:0E0000000C947A000C9400000C9400000C94F8
:10000E0000000C9400000C9400000C9400000C9462
:10001E0000000C9400000C9400000C9400000C9452
:10002E0000000C9400000C9400000C9400000C9442
:10003E0000000C94DC000C9400000C94A9000C94AD
:10004E0000000C9400000C9400000C9400000C9422
:10005E0000000C9400000C9400001027E8036400CC
:10006E000A00010000100001100001000000000055
:10007E000A00000000000000000000000000000068
:10008E000000000000000000000000000000000062
:10009E000000000000000000000000000000000052
:1000AE000000000000000000000000000000000042
:1000BE000000000000000000000000000000000032
:1000CE00000A0A0A0A0A0A0A0A0A0A0A0A0A0A0A8C
:1000DE000A00020002007A00020004007C00010007
:1000EE0007037E000000F894EE27EFBBF1E0F5BFAA
:1000FE00E5BF8DE0A2E0BB27ED938A95E9F780E09E
:10010E0098E0A0E0B1E0ED930197E9F7E0EEF0E0C2
:10011E0085919591009761F0A591B59105901590F7
:10012E00BF01F00105900D920197E1F7FB01F0CFB1
:10013E00E8E0EEBBEFEFEDBFE8E0EEBFC0E0D3E0EE
:10014E000C940204AA93EA93FA93EFB7EA931A93E4
:10015E000A931091C0000091C600E12FEC71E9F4F2
:10016E00E0911804EF5FE0931804E150F0E0E150E5
:10017E00FC4F0083A0911804A93119F4E0E0E0933C
:10018E001804A0911A04AF5FA0931A04A93129F4A0
:10019E00E0E0E0931A04689437F809911991E99117
:1001AE00EFBFF991E991A99118950A921A926A9363
:1001BE007A938A939A93AA93BA93EA93FA93EFB7A0
:1001CE00EA93E0915503F09156033196E09355036F
:1001DE00F09356030E945131E1E5F1E00E943F3E5B
:1001EE000E2E0E945131E3EAF2E00E943F3EE029DA
:1001FE0009F444C2A0915303B0915403E5E0F0E03A
:10020E000E94633E0E2EA0912803EEE00E94353E22
:10021E00E02121F0E0912803EF5F03C025FC03C02D
:10022E00E0E0E0932803A0912803AE3011F4689427
:10023E0025F8A0913203A13029F4F79B02C0F7985C
:10024E0001C0F79AE1E02E260E9456310E945F31DE
:10025E00E093E303F093E4036093E5037093E60306
:10026E000E946631A7ECB3E00E946B310E9472319E
:10027E00AFEEB3E00E946B310E9477310E94803165
:10028E000E945D3DE093C703F093C8036093C903DA
:10029E007093CA03A091EF03B091F0038091F10324
:1002AE009091F203E0E0F0E060E772E40E945D3DC1
:1002BE00E093EF03F093F0036093F1037093F20376
:1002CE000E9485310E948A310E2E0E948F310E942B
:1002DE008A31E02161F1E091EF03F091F00360913A
:1002EE00F1037091F2030E9477310E945D3DE0931D
:1002FE00EB03F093EC036093ED037093EE030E9417
:10030E009431A7E6B3E00E949D31A091EB03B0912A
:10031E00EC038091ED039091EE030E945F31E09328
:10032E00CF03F093D0036093D1037093D2030E9456
:10033E00A2310E94AB310E94B4310E94BF3CE093C7
:10034E00D703F093D8036093D9037093DA030E9416
:10035E00A2310E94BD310E94C23D0E2E0E94C231BA
:10036E00E8EEFDEF0E945D3EE021D1F00E94A23149
:10037E000E94AB31A091F703B091F8038091F9037D
:10038E009091FA030E94C731E093F703F093F803BC
:10039E006093F9037093FA03A5E7B3E00E949D31D1
:1003AE000E94A2310E94AB310E94CC310E94BF3C10
:1003BE00E093FB03F093FC036093FD037093FE0345
:1003CE000E94D5310E94DE310E94C731AFEAB3E000
:1003DE000E944E3C0E94593F0E94D531AAE0B0E0E7
:1003EE0080E090E00E94993E0E94CC310E94833CB6
:1003FE000E94A23D70F0E0E0E093FB03E093FC036B
:10040E00E093FD03E093FE030E94F13131960E94CA
:10041E00F631E091B303F091B4036091B50370919E
:10042E00B6030E94A2310E940F3DDF01CB010E9454
:10043E005F31E093E703F093E8036093E903709371
:10044E00EA030E94FB310E94BF3C0E940432E091FD
:10045E000E03F0E00E940D320E940D3E0E94993E66
:10046E00DF01CB01E091F303F091F4036091F5030A
:10047E007091F6030E94723F0E94C731A9E8B3E063
:10048E000E9416320E9456310E94C33F3CF5A09145
:10049E00E703B091E8038091E9039091EA030E948B
:1004AE001B327F936F93FF93EF93A091E303B09171
:1004BE00E4038091E5039091E6030E941B32AF9115
:1004CE00BF918F919F910E945D3DE093DF03F0936A
:1004DE00E0036093E1037093E20309C0E0E0E09370
:1004EE00DF03E093E003E093E103E093E203A091E6
:1004FE00E203AA23AAF40E942232E0E0F0EC69E7BC
:10050E0074EC0E94A23D18F40E942B3208C00E9487
:10051E0032320E94193CA1E9B3E00E94163214C097
:10052E000E942232E0E0F0EC69E774E40E94A23D02
:10053E0009F008F403C00E942B3206C00E9432322A
:10054E00A1E9B3E00E9416320E943B320E9444326F
:10055E000E94BF3C0E944D32E091C703F091C80348
:10056E006091C9037091CA030E9456320E94A23D47
:10057E0068F5E091CF03F091D0036091D1037091B3
:10058E00D2030E9456320E94BF3CE093CB03F093FD
:10059E00CC036093CD037093CE030E9456320E941B
:1005AE005F320E94B83CDF01CB010E9494310E9461
:1005BE005D3DA0E0B0E081E695E40E940F3DA5E828
:1005CE00B3E00E941632689424F802C0E0E12E26B1
:1005DE000E943B320E9468320E94BF3CE093D303DC
:1005EE00F093D4036093D5037093D6030E946832C0
:1005FE00E0E0F0E060E87FE30E94A23D09F008F43D
:10060E0012C0E093D303E093D403E093D503E093B9
:10061E00D6030E947132EF5FFF4F6F4F7F4F0E94E4
:10062E007A320E9483320E948932A034E2E4BE07FD
:10063E00EFE08E07E0E09E0778F0E0E0E0937703CE
:10064E00E0937803E0937903E0937A03AFE5B0E0AB
:10065E000E94BD310E94983F0E9444320E94923205
:10066E00A7E5B3E00E949D31A0912603AC3308F4B8
:10067E00F298A0912603AC3309F4F29A0E945131FC
:10068E00A33AE2E0BE0709F08DC0A09125030E94B7
:10069E0096320E949B320E94BD310E94693E0E949A
:1006AE00A432E02191F0E0912603EF5FE093260360
:1006BE00E0912503F0E03296A0912603B0E0EA1710
:1006CE00FB0719F4ECE3E0932603E0E0E093550317
:1006DE00E0935603D394A0910F03A13028F4E09138
:1006EE000F03EF5FE0930F030E94AB32E8E5F2E0F9
:1006FE000E945D3E0E2E0E94B032E02199F0E091F4
:10070E006B03F0916C033196E0936B03F0936C03E3
:10071E000E94AB320E94B532EA1BFB0BE0937103D1
:10072E00F0937203ECE3ED1589F4DD24C394EC151C
:10073E0069F4CC24E0910003EF5FE0930003A091F5
:10074E000003A43119F4E0E0E0930003A0912D031F
:10075E00A130D0F0E0911203EF5FE0931203A0916D
:10076E001203A23088F0E0911103EF5FE0931103C2
:10077E00E0E0E0931203E0912D03A0911103EA173C
:10078E0018F4E0E0E0931103E0912D03E03019F44A
:10079E00E0E0E0931103A0912D03A23019F4E1E003
:1007AE00E0931103E991EFBFF991E991B991A99104
:1007BE009991899179916991199009901895AA93B7
:1007CE00E881E066E0937C0085E28A95F1F7E0919E
:1007DE007A00E064E0937A00E0917A00E071E1F350
:1007EE00E0917A00E061E0937A00E0917800F09178
:1007FE00790021960895EF97A0978FE5A0E0B0E0DD
:10080E00E0E8F0E00E94D83FFF2411E001E0E0E8CC
:10081E00E0936100E0E0E0936100EFE0E4B9E1E035
:10082E00E5B9E0E0E7B9E4E0E8B9EAEFEAB9E7EE06
:10083E00EBB9E0E0E4BDE3E0E5BDE0E0E6BDE7BD39
:10084E00E8BDE0938000E0938100E0938500E093A3
:10085E008400E0938700E0938600E0938900E093A4
:10086E008800E0938B00E0938A00E093B600E1EA03
:10087E00E093B000E2E0E093B100E0E0E093B2007C
:10088E00E093B300E093B400E1E0E0936E00E0E0AB
:10089E00E0936F00E0937000E0936900EDBBE0938E
:1008AE006800E093C000E8E9E093C100E6E0E09361
:1008BE00C200E0E0E093C500E7E4E093C400E0E8A6
:1008CE00E0BFE0E0E0937F00E0937E00E0E6E0939F
:1008DE007C00E6E2E0937A00E0E0E0937B00ECBD82
:1008EE00E093BC0078945F9A0E94BA320E94BE32A6
:1008FE000E94C4320E94CB320E94D8320E94BA3279
:10090E00EAE06E16B8F5ABE3B0E00E94E532A6E27F
:10091E00B0E0E0E00E94A83FA7E2B0E00E94A83F4E
:10092E00A6E3B0E00E94A83FA7E3B0E00E94A83F74
:10093E00A8E3B0E00E94A83FA1E5B0E0E8EEF3E046
:10094E000E94A03FA3E5B0E00E94E532A5E5B0E02D
:10095E000E94E532A7E5B0E00E94E532A9E5B0E0DD
:10096E000E94E532ABE5B0E00E94E532ADE5B0E0C5
:10097E000E94E532EAE09E1650F4A1E4B0E00E9437
:10098E00E532A9E4B0E00E94E532689426F8EAE088
:10099E00BE1618F4689430F827F8689433F8EBE133
:1009AE00E09316030E94EA32E8ECF0E00E94F13286
:1009BE00E0EDF7E00E94F632E8ECF0E0E0937F0322
:1009CE00F0938003A0E0B0E00E948C3FE093170309
:1009DE00A1E0B0E00E948C3FEFA3A2E0B0E00E9445
:1009EE008C3FE0931803A3E0B0E00E948C3FE093AD
:1009FE001A03A4E0B0E00E948C3FE9AFA5E0B0E09E
:100A0E000E948C3FEAAFA6E0B0E00E948C3FEBAFB5
:100A1E00A7E0B0E00E948C3FE0931B03A8E0B0E09B
:100A2E000E948C3FE0931C03F798F198AAE0B0E087
:100A3E000E948C3FE0932503A9E3B0E00E94883F1B
:100A4E000E94FB32A2E1B0E00E948C3FEDABA3E12D
:100A5E00B0E00E948C3FEEABA4E1B0E00E948C3F70
:100A6E00EFABABE0B0E00E948C3FE9ABACE0B0E0A6
:100A7E000E948C3FEAABADE0B0E00E948C3FEBAB46
:100A8E00ADE3B0E00E94883FEF8FF8A3AEE0B0E098
:100A9E000E948C3FE0933303AFE0B0E00E948C3FA6
:100AAE00E0933503A0E1B0E00E948C3FE093340365
:100ABE00AFE5B0E00E94843F0E947A32ABE3B0E033
:100ACE000E94883FA3ECB3E00E9400330E945F3285
:100ADE00A7E5B3E00E949D310E9444320E94073385
:100AEE000E944D32A1E1B0E00E948C3FF0E0EF8B0E
:100AFE00F88FAFE3B0E00E94883FEBA3FCA3AFE416
:100B0E00B0E00E94883FE98FFA8FA1E4B0E00E9426
:100B1E00883FA7EDB3E00E940033A9E4B0E00E9445
:100B2E00883FA3EFB3E00E9400330E94FB310E9486
:100B3E0007330E940432A3E4B0E00E94883F0E9473
:100B4E000B33A7E4B0E00E94883F0E940D3E0E9446
:100B5E001033A5E1B0E00E948C3F0E94D33F23F8F2
:100B6E00A5E4B0E00E94883F0E941933A6E1B0E0F0
:100B7E000E948C3FE0930603A7E1B0E00E948C3FF9
:100B8E00E0930803A8E1B0E00E948C3FE0930903D4
:100B9E00A9E1B0E00E948C3FE0930A03AAE1B0E025
:100BAE000E948C3FE0930B03ABE1B0E00E948C3FC0
:100BBE00E0930C03ACE1B0E00E948C3FE09329037C
:100BCE00ADE1B0E00E948C3FE0932A03AEE1B0E0CD
:100BDE000E948C3FE0932B03AFE1B0E00E948C3F6C
:100BEE00E0932C03A0E2B0E00E948C3FE0932D0333
:100BFE00A1E2B0E00E948C3FE0932E03A2E2B0E0AF
:100C0E000E948C3FE0932F03A3E2B0E00E948C3F42
:100C1E00E0933003ABE4B0E00E94883F0E94F631CF
:100C2E00A4E2B0E00E948C3FE0930E03A5E2B0E098
:100C3E000E948C3F0E94D33F36F8A8E2B0E00E949B
:100C4E008C3FE0931003A9E2B0E00E948C3FECA72A
:100C5E00ADE4B0E00E94883FEB8FFC8FAAE2B0E0DB
:100C6E000E948C3FE0934103ABE2B0E00E948C3FC8
:100C7E00E0934203ACE2B0E00E948C3FE09343036A
:100C8E00ADE2B0E00E948C3FE0931D03AEE2B0E017
:100C9E000E948C3FE0931F03A9E0B0E00E948C3FBE
:100CAE00E0932003AFE2B0E00E948C3FE09321037B
:100CBE00A0E3B0E00E948C3FE0932203A1E3B0E0FA
:100CCE000E948C3FE0931503A2E3B0E00E948C3F9C
:100CDE00E0934A03A3E3B0E00E948C3FE0934B0302
:100CEE00A4E3B0E00E948C3FE0934C03A5E3B0E098
:100CFE000E948C3FE0934E030E941E33E0937503D7
:100D0E00F09376030E941E33A7EFB3E00E940033E8
:100D1E0036FE0BC0A6E2B0E00E948C3FCE2EA7E2BC
:100D2E00B0E00E948C3FE0930003E1E0E0933F03CC
:100D3E00A0910203AE3128F4E0910203EF5FE0933D
:100D4E000203A0910203AE3189F4E0E0E093380390
:100D5E00E0939903E0939A03EBE0F0E00E942333D3
:100D6E00E8EB0E942833E4E1E0930203ECA5E030C7
:100D7E0041F5A091FF03ECE30E94173E0E2EA091C9
:100D8E000004E7E00E94173E0E22A0911804EBE04B
:100D9E000E94173EE02169F0E0910104E0933703D1
:100DAE00E0910204E09338030E942E33E0E0E093DA
:100DBE000203A0911804AC3020F00E943C330E9434
:100DCE004833ACA5A130E9F4A091FF03E8E20E94FC
:100DDE00173E0E2EA0911804E8E00E94173EE02167
:100DEE0041F0E1E0E09337030E942E33E0E0E09320
:100DFE000203A0911804AC3020F00E943C330E94F4
:100E0E004833ACA5A33009F079C0A091FF03ECE6FE
:100E1E000E94173E0E2EA0910004EBE00E94173E9A
:100E2E000E22A0911804EFE00E94173EE02109F473
:100E3E0041C0E0910204E0933703E0910304E09394
:100E4E003803E0910404F0E00E945433F0919903CA
:100E5E00E0E00E945433E0910504F0E0A091990384
:100E6E00B0919A03EA0FFB1F0E945433E0910604DF
:100E7E00E0934803E0910904E0934703E0910A04EC
:100E8E00F0E00E942333E0910B04E0933903E091EC
:100E9E000704F0E0E0939B03F0939C03E0910804B9
:100EAE00F0E0E0939D03F0939E03E0E0E0931804DE
:100EBE00E0930203A0911804A03100F1E0E0E0936A
:100ECE00FF03E0930004E0930104E0930204E09337
:100EDE000304E0930404E0930504E0930604E09316
:100EEE000704E0930804E0930904EBE0E0930A049E
:100EFE00E8EBE0930B04E0E0E0931804E8EC5E16F8
:100F0E0030F45394EEE1E51511F4E1E04E2E0E941B
:100F1E005933E7EAE0937A00A6E00E945D33EB8B4B
:100F2E00FC8BE7E2E0937A000E9459330E94BE32B6
:100F3E000E94023E0E94FE3DED8BFE8BE7E2E093A7
:100F4E007A000E9459330E9464333B9780F1A0E0EF
:100F5E000E945D33662777270E946D33A8EEB3E0BB
:100F6E0080E090E00E94C43EDF01CB010E9472330C
:100F7E00662777270E94063F0E946D33A3EBB3E0EE
:100F8E000E94853C0E94593FE0910703EF5FE0937A
:100F9E000703E0910603A0910703AE1730F00E94FD
:100FAE007733EC87FD876E877F87E894F3F80E948E
:100FBE007C330E94BE320E94C4320E948333A2E070
:100FCE000E945D33DF01E5E0F0E00E94C93E8E2E07
:100FDE000E947C330E94D8328AE48A95F1F70E94EF
:100FEE00CB320E9483330E948A330E947C33E7EA1D
:100FFE00E0937A00A5E0E3DBEF2FF0E0EDA3FEA394
:10100E000E947C330E946433AE2E0E947C33A091EA
:10101E004E03A13069F4EDA1FEA1ADA1BEA10E94C7
:10102E00913EDF01E6EDF0E00E94C93EEDA3FEA386
:10103E00E0911003E03009F0A0C0E1E0E515B1F554
:10104E000E9494335E9710F4E1E0EFA70E94943370
:10105E000E9499330E949433EAEFF0E00E945D3EC5
:10106E00E02111F0E2E0EFA70E949433AB3FE0E005
:10107E00BE0710F0E3E0EFA7ADA1BEA15E9710F49E
:10108E00E1E0EEA70E949F33ADA1BEA1EAEFF0E032
:10109E000E945D3EE02111F0E2E0EEA7ADA1BEA1FF
:1010AE00AB3FE0E0BE0710F0E3E0EEA70E94943302
:1010BE000E94A233AFA50E94AD3311F0E4E009C047
:1010CE000E9494330E94B233AFA50E94AD3311F04B
:1010DE00E5E0EFA7ADA1BEA10E94A233AEA50E948E
:1010EE00AD3311F0E4E009C0ADA1BEA10E94B23350
:1010FE00AEA50E94AD3311F0E5E0EEA7AFA50E94BC
:10110E009632AFA50E94BD3369F0EDA1FEA10E94FB
:10111E00C233E8E2F0E0EDA3FEA3AA89AC3511F4E8
:10112E000E94C733AFA50E94CD33AFA5E5E00E9464
:10113E00173EE02911F00E94C733AEA50E949632E9
:10114E00AEA50E94BD3369F0E8E2F0E0EDA3FEA388
:10115E00AFA50E949632AFA50E94BD3311F00E943A
:10116E00C733AEA50E94CD330E94D233E02921F0C1
:10117E00ECE3F0E0EDA3FEA303C0E0E0EFA7EEA7E3
:10118E00ADA1BEA1A73DE0E0BE0720F0E6EDF0E088
:10119E00EDA3FEA30E94D7330E94DD330E94353E9D
:1011AE00E021E9F1E4E1EAA76894F3F80E94E7335D
:1011BE000E94ED3319F0E1E0E0931403A12F0E9499
:1011CE00F6330E94FB3321F0F398F49A12E01CC020
:1011DE00A12FE2E00E94173E0E2E0E94FB3359F023
:1011EE00F498F59AABADA13010F013E003C0F5986A
:1011FE00F39A11E009C0A12F0E94FE330E94FB3327
:10120E0019F0F598F39A11E0A62DE9E00E943A3E06
:10121E000E2E0E94ED3319F0E0E0E0931403E091FE
:10122E004F03E09340030E949433D39708F45DC0BC
:10123E000E9403340E940834E12F0E940F3420F0E4
:10124E00E8ECF0E00E94C233A0914203A13011F409
:10125E000E941F34E12F0E942A340E943A34AC912E
:10126E00A13008F441C00E9441340E944A340E94C9
:10127E00CE3F4CF40E943A340E9456340E94CE3D2A
:10128E000E94603423C00E9469340E946B34EF9335
:10129E000E9469340E947434AF91EA2379F00E945F
:1012AE003A340E9456340E94D33DA093A303B093C8
:1012BE00A4038093A5039093A60308C00E946934EB
:1012CE000E947D341CF00E9487340EC0A091A303AF
:1012DE00B091A4038091A5039091A6030E94963429
:1012EE000E94063F0E94C23304C00E94C7330E9470
:1012FE0087340E94E7330E949B340E220E94A03452
:10130E0001F10E9494330E94BF3F10F4E4E1E8A77C
:10131E00A09127030E9496320E94A434E02141F04E
:10132E00E3E0E0933603E0E0E09327030E94AA3463
:10133E00E0914F03E09327036894F0F821F8E894C6
:10134E00F4F8A0912F03A130D9F50E94B0340E2EDF
:10135E00A0914003E0E50E94353E0E22A0912703A6
:10136E00E8EC0E94353E0E94B2340E22A0E0F4FC5E
:10137E00A1E00E94BA3429F0E0912703EF5FE093D9
:10138E0027030E949F33ADA1BEA1E0E5F0E00E94CD
:10139E005D3E0E22A0912703E0E00E943A3E0E949D
:1013AE00B234E02169F0E0912703E150E093270386
:1013BE000E94BF340E94C33419F0E3E00E94C93486
:1013CE000E94A4340E94CC34A09127030E94AD3316
:1013DE0021F0E0E0E093280306C0A0912803A2309C
:1013EE0010F4E89425F8A0912703A13020F0E091A5
:1013FE002703F0E002C00E940334E0935303F093FE
:10140E0054030E940334309729F4E89421F8689429
:10141E00F4F827C00E94D5340E2E0E94B0340E224E
:10142E00A0912F030E94AD331E2EA09127030E9480
:10143E0096320E94D5340E22A0914003EFE40E9412
:10144E003A3E0E22A0912F030E94BA34E12949F0B0
:10145E00E0E0E09327030E94C733E89422F86894F3
:10146E0021F8E09104030E949433F0E0EA17FB07A1
:10147E0020F4E0914F03E09304030E94DC340E94B9
:10148E00893E0E22A09133030E94AD331E2E0E9480
:10149E00DC340E94813E0E22A09134030E94AD33B3
:1014AE00E12961F0E0914F03E09304030E94BF3401
:1014BE000E94EB3419F0E2E00E94C934A091270398
:1014CE00A13080F0689422F80E940334A091270383
:1014DE00B0E0AE17BF0728F0E0912703F0E00E94BE
:1014EE00C23302C0E89422F80E94EF340E22A0E02C
:1014FE0031FCA1E00E94AD3331F0689431F80E94C6
:10150E0003340E94F1320E94EF34E02151F10E9427
:10151E0001350E94093594F0A885B985EF8DF8A1A3
:10152E00EA1BFB0BA3E0B0E00E94BF3E0E94113508
:10153E00AE1BBF0BA0938103B09382030E940135B3
:10154E000E94C33F2CF40E94163532970E94F1324E
:10155E00A0918203AA232AF4E0E0E0938103E093B2
:10156E0082030E941B350E94C93F74F50E941B35F1
:10157E000E94D33D0E94093564F0AF8DB8A1E88575
:10158E00F985EA1BFB0B0E941135EA0FFB1F0E9427
:10159E00F1320E941B350E94D33DA230E0E0BE071F
:1015AE00E0E08E07E0E09E072CF00E9416353196A3
:1015BE000E94F1320E941135AB3FE0E0BE0724F0ED
:1015CE00EAEFF0E00E94F1320E9416350E94943349
:1015DE00AE17BF0710F4E89431F80E9416350E943A
:1015EE009433EA17FB0720F40E9416350E94C2338B
:1015FE000E942435A0E032FCA1E00E9430350E940A
:10160E00C33431F0689432F80E9435350E94F632B8
:10161E000E9424350E94C334A1F10E943A35DF01A5
:10162E00CB01E0E0F0E060E070E40E94A23D09F042
:10163E0008F414C00E943A35A0E0B0E080E890E4CF
:10164E000E940F3D0E9443350E94123E0E94743F3D
:10165E000E94C731A3E8B3E00E9416320E943A35C9
:10166E000E94B93F2CF40E94483535970E94F632FD
:10167E00A0918403AA232AF4E0E0E0938303E0938D
:10168E008403EF89F88D0E944D350E9450350E94DB
:10169E00C23D0E2E0E94C334A9F10E945535DF01C2
:1016AE00CB01E0E0F0E060E470E40E94A23D09F0BE
:1016BE0008F414C00E945535A0E0B0E080EA90E432
:1016CE000E940F3DDF01CB010E9448350E945E351E
:1016DE000E94BF3CA3E8B3E00E9416320E9455352B
:1016EE000E94B93F2CF40E94483535960E94F6327E
:1016FE000E944335A53CE9E0BE0724F0E4ECF9E096
:10170E000E94F6320E943535DF010E9448350E9454
:10171E005D3E0E2E0E94C33411F0E89432F80E9402
:10172E003535DF010E9448350E94633E0E2E0E9421
:10173E00C33421F00E9443350E9463350E94683500
:10174E000E94893E0E2EA0E034FCA1E00E94AD3333
:10175E0031F0689434F80E9435350E946E350E943F
:10176E0068350E94C93F54F50E9473350E940935B1
:10177E0094F0EFA1F0E0A091AB03B091AC03AE1BDF
:10178E00BF0BE3E0F0E00E947B35AE1BBF0BA093D6
:10179E008B03B0938C030E9473350E94C33F2CF4CD
:1017AE000E94823532970E946E35A0918C03AA2337
:1017BE002AF4E0E0E0938B03E0938C030E946835FB
:1017CE000E94CE3F84F50E948735A430E0E0BE072C
:1017DE00E0E08E07E0E09E0784F0AFA1BB27E0912A
:1017EE00AB03F091AC03AE1BBF0BE2E0F0E00E9446
:1017FE007B35EA0FFB1F0E946E350E9487350E94D3
:10180E00C33F2CF40E94823532960E946E35A09111
:10181E008B03B0918C03A53CE9E0BE0724F0E4EC09
:10182E00F9E00E946E350E943535DF010E94823547
:10183E00AE17BF0710F4E89434F80E943535DF0177
:10184E000E948235EA17FB0730F4A0918B03B0910A
:10185E008C030E946335E09113030E949433F0E0F1
:10186E00EA17FB0720F4E0914F03E0931303E09196
:10187E001303F0E035970E9494330E945D3E6E2F65
:10188E000E2EA0E031FCA1E00E94BA341E2E062ED0
:10189E00A0E032FCA1E00E94BA341E2A062EA0E07F
:1018AE0034FCA1E00E94BA34E12961F0E0914F03CB
:1018BE00E09313030E94BF340E94C33419F0E2E098
:1018CE000E94C934A0913603A13078F00E94C7332C
:1018DE00A0913603A13021F4EAE0F0E00E94C23379
:1018EE00E0913603E150E09336030E949F33A091BE
:1018FE002F030E94AD331E2EADA1BEA1E0E5F0E098
:10190E000E94633E0E2EA0912F03E1E00E94173E2F
:10191E000E94B234E0211E2A0E949F33A0912F0311
:10192E00E1E00E94173E0E220E94EB34E129E9F01D
:10193E00E0E0E0930503A0912703A13018F0E2E068
:10194E00E0933603E0E0E0932703EDA1FEA1F297CA
:10195E000E945035A6EFB8E28CE99FE30E940F3D3E
:10196E00DE0195960E949D3103C0E0E0EDA3EEA34B
:10197E000E940334ED8FFE8F0E9496350E2EA0919D
:10198E002A030E94BA3411F0299A01C029980E94A4
:10199E0096350E2EA0914103E2E00E94173EE02103
:1019AE0011F0EFEF01C0E0E0E09344030E94E73353
:1019BE000E949B34E02119F0EDA1E0934D03A0911C
:1019CE004D03A13068F0E0914D03F0E0EDA3FEA3CE
:1019DE000E9494330E94BF3F18F4E0E0E0934D0361
:1019EE00A82DE4E60E94353E6E2F0E2E0E949935EC
:1019FE000E22AA89EDE50E941C3E0E94A0351E2EE5
:101A0E00062E0E9499350E220E949B34E0211E2A3A
:101A1E000E94B5320E94AB320E943F3E0E94A73513
:101A2E000E94B032E021E12941F1E0915703F0919B
:101A3E005803ABE3B0E00E94AF350E94B5350E946B
:101A4E00FB310E9492320E94C2350E94C735EC2DA6
:101A5E00A6E2B0E00E94CB35E0910003A7E2B0E031
:101A6E000E94CB350E94D1350E94BA325F98A8EE03
:101A7E00B3E00E940F3C5F98FECFAB2D0E94DA358B
:101A8E000E949B34E02131F0E894F2F827F8E0E070
:101A9E00E0933D030E94DF350E949B34E02171F0FC
:101AAE00E0913D03EF5FE0933D03A0913D03AA302B
:101ABE0029F4E0E0E0933D03E09332030E94DF352A
:101ACE00A0E0F2FCA1E00E9430350E949B34E021A0
:101ADE00C1F1E4E1E9A76894F2F8E0913203EF5F17
:101AEE00E0933203A09132030E94FE330E94A03491
:101AFE0019F0E1E0E0933203A09132030E94CD335E
:101B0E000E94A03419F0E2E0E0933203A091320378
:101B1E000E94FE33A0912A030E9430350E94C334E6
:101B2E0019F0E1E0E0933203A09132030E94CD332D
:101B3E00A0E0F0FCA1E00E94BA3419F0E3E0E093DB
:101B4E003203E0913203E03041F4F7982A98E0E056
:101B5E00E0934503E093460322C0A0913203A130E7
:101B6E0031F42A98EFE7E0934503E0E015C0A09129
:101B7E003203A23039F4F79A2A98EFE7E09345033F
:101B8E00E0E00AC0A0913203A33059F4F79A2A9AE2
:101B9E00EFE7E0934503EFEFE0934603E1E0E093D8
:101BAE003103A0914403AF3F19F4EFEFE0934503E7
:101BBE000E94E835E081E093B4000E94B0340E2E0E
:101BCE000E9496350E220E94EB341E2E0E94A434E3
:101BDE000E94CC34A62DEAE00E94353E0E22A02FA4
:101BEE00E3E60E941C3EE021E129C9F1A091290300
:101BFE00A13009F45C9AE0910303EF5FE0930303D5
:101C0E00A0912903A33029F4E27011F45C9801C06D
:101C1E005C9AA0910303E5E00E943A3E0E2EE4E1A9
:101C2E000E94353EE02199F0E0910303E170AFEFA1
:101C3E00EA02F001E093B400A0912903A23039F436
:101C4E00E0910303E17011F45C9801C05C9AA091DD
:101C5E000303A03118F0E0E0E093030325C05C9885
:101C6E00A0E030FCA1E00E94F633A09132030E9466
:101C7E00AD33D1F0E0913C03EF5FE0933C03A091D4
:101C8E003C03A13019F4EFEFE093B400A0913C03B4
:101C9E00A33019F4E0E0E093B400A0913C03A4302B
:101CAE0019F4E0E0E0933C030E94EE350E94F53516
:101CBE00E1F0E0911C03A0911E03AE1728F4E09111
:101CCE001E03EC5FE0931E03E0911C03A0911E0324
:101CDE00EA1728F4E0911E03E250E0931E03033648
:101CEE0021F4E0911C03E0931E030E94EE35EA17E7
:101CFE00FB07E0F4E0911D03A0911E03AE1728F43C
:101D0E00E0911E03EC5FE0931E03E0911D03A09192
:101D1E001E03EA1728F4E0911E03E250E0931E031F
:101D2E00033621F4E0911D03E0931E03E0911E03A0
:101D3E00E093B300EAE0E91518F4E894F1F826F818
:101D4E000E94FE35A0E026FCA1E00E943035A0E006
:101D5E00F1FCA1E00E9430350E949B34E02139F164
:101D6E006894F1F8E0910D03EF5FE0930D03E0E06E
:101D7E00EDA7ADA5A53088F40E940436A081A13050
:101D8E0018F0E5E0EDA705C0E0910D03EF5FE093DD
:101D9E000D03EDA5EF5FEDA7ECCFA0910D03A530E0
:101DAE0018F0E0E0E0930D030E94043600810E94DB
:101DBE00FE35A0912403EFEF0E94353EE02121F085
:101DCE00E0912403EF5F03C0E894F1F8E0E0E093C4
:101DDE002403A0912403A43109F086C1AA89E0E06E
:101DEE000E942B3E0E2E0E949B34E02119F0EA89B0
:101DFE00E150EA8B033610F403E676C101E0E0E031
:101E0E00E0930D03E0911703A0E0B0E00E94CB3504
:101E1E00EFA1A1E0B0E00E94CB35E0911803A2E063
:101E2E00B0E00E94CB35E0911A03A3E0B0E00E942F
:101E3E00CB35E9ADA4E0B0E00E94CB35EAADA5E02C
:101E4E00B0E00E94CB35EBADA6E0B0E00E94CB3502
:101E5E00E0911B03A7E0B0E00E94CB35E0911C039C
:101E6E00A8E0B0E00E94CB35E0912003A9E0B0E0FD
:101E7E000E94CB35E0912503AAE0B0E00E94CB355D
:101E8E000E947233A9E3B0E00E94AF35EDA9A2E142
:101E9E00B0E00E94CB35EEA9A3E1B0E00E94CB35B5
:101EAE00EFA9A4E1B0E00E94CB35E9A9ABE0B0E028
:101EBE000E94CB35EAA9ACE0B0E00E94CB35EBA98D
:101ECE00ADE0B0E00E94CB35EF8DF8A1ADE3B0E010
:101EDE000E94AF35E0913303AEE0B0E00E94CB3507
:101EEE00E0913503AFE0B0E00E94CB35E0913403D2
:101EFE00A0E1B0E00E94CB35EF89A1E1B0E00E94F5
:101F0E00CB35EBA1FCA1AFE3B0E00E94AF35E98D7C
:101F1E00FA8DAFE4B0E00E94AF350E94B5350E9455
:101F2E000A36A3E4B0E00E94AF35E0917B03F09156
:101F3E007C03A7E4B0E00E94AF35E0E023FCE1E0D3
:101F4E00A5E1B0E00E94CB350E94B532A5E4B0E029
:101F5E000E94AF35E0910603A6E1B0E00E94CB35BA
:101F6E00E0910803A7E1B0E00E94CB35E0910903B0
:101F7E00A8E1B0E00E94CB35E0910A03A9E1B0E000
:101F8E000E94CB35E0910B03AAE1B0E00E94CB3565
:101F9E00E0910C03ABE1B0E00E94CB350E94FB3127
:101FAE000E9492320E94C235E0912903ACE1B0E06A
:101FBE000E94CB35E0912A03ADE1B0E00E94CB3513
:101FCE00E0912B03AEE1B0E00E94CB35E0912C0303
:101FDE00AFE1B0E00E94CB35E0912D03A0E2B0E07E
:101FEE000E94CB35E0912E03A1E2B0E00E94CB35EA
:101FFE00E0912F03A2E2B0E00E94CB35E0913003D6
:10200E00A3E2B0E00E94CB350E94C735E0910E03EB
:10201E00A4E2B0E00E94CB35E0E036FCE1E0A5E2C0
:10202E00B0E00E94CB35E0911003A8E2B0E00E9430
:10203E00CB35ECA5A9E2B0E00E94CB35EB8DFC8D43
:10204E00ADE4B0E00E94AF35E0914103AAE2B0E00A
:10205E000E94CB35E0914203ABE2B0E00E94CB355B
:10206E00E0914303ACE2B0E00E94CB35E0911D035A
:10207E00ADE2B0E00E94CB35E0911F03AEE2B0E0DE
:10208E000E94CB35E0912103AFE2B0E00E94CB3548
:10209E00E0912203A0E3B0E00E94CB35E09115035E
:1020AE00A1E3B0E00E94CB350E948332A1E0B0E004
:1020BE000E940F3CE0914A03A2E3B0E00E94CB35B0
:1020CE00E0914B03A3E3B0E00E94CB35E0914C03CB
:1020DE00A4E3B0E00E94CB35E0914E03A5E3B0E05F
:1020EE000E94A83FE1E04E2E0E94FE35A0E0F1FCDA
:1020FE00A1E00E943035AA89E4E60E94263E0E94A5
:10210E00A03551F06894F1F8EA89EF5FEA8BAA895D
:10211E00A43611F4E0E0EA8BEAE0E61510F4E89458
:10212E00F0F80E94E733A0E0F0FCA1E00E94303509
:10213E00AA89E0E00E94213E0E94A03551F06894E9
:10214E00F0F8EA89E150EA8BAA89AF3F11F4E3E691
:10215E00EA8B0E94D7330E940F36C1F00E941536CB
:10216E00A9F4A0913A03A43119F4E7E0E0933A03FD
:10217E00E0E0E0933B03E894F3F8A0913A03A33038
:10218E0028F0E0913A03E150E0933A03AB2DEAE0F8
:10219E000E94353E0E2E0E940F36C1F00E9415365B
:1021AE00A9F4A0913A03A43119F4E7E0E0933A03BD
:1021BE00E0E0E0933B03E894F2F8A0913A03A330F9
:1021CE0028F0E0913A03E150E0933A03AB2D0E94E0
:1021DE00DA35AA2DEAE00E943A3EE02131F0E0E045
:1021EE00E0933B03E4E1E0933A03EAE0EA1510F4EE
:1021FE00E894F3F80E94D7330E94DD330E94173E15
:10220E00E02109F42AC36894F3F8AA89A13049F4AD
:10221E00A0911703A13028F4E0911703EF5FE0932C
:10222E001703AA89A23031F4AFA1AF3518F4EFA18C
:10223E00EF5FEFA3AA89A33049F4A0911803A63942
:10224E0028F4E0911803EF5F0E942036AA89A4308B
:10225E0049F4A0911A03A83228F4E0911A03EF5F13
:10226E00E0931A03AA89A53031F4A9ADA43618F467
:10227E00E9ADEF5FE9AFAA89A63031F4AAADA43675
:10228E0018F4EAADEF5FEAAFAA89A73031F4ABAD2F
:10229E00A43618F4EBADEF5FEBAFAA89A83049F482
:1022AE00A0911B03AF3F28F4E0911B03EF5FE09377
:1022BE001B03AA89A93049F4A0914103AF3F28F42A
:1022CE00E0914103EF5FE0934103AA89AA3049F4FC
:1022DE00A0914203AF3F28F4E0914203EF5FE093F9
:1022EE004203AA89AB3049F4A0914303AF3F28F4CF
:1022FE00E0914303EF5FE0934303AA89AC3049F4C6
:10230E00A0910E03A03328F4E0910E03E45FE09356
:10231E000E03AA89AD3069F4A0915903B0915A0306
:10232E00A43CE9E0BE0728F40E94723331960E9465
:10233E00FB32AA89AE3031F4ADA9A43618F4EDA95A
:10234E00EB5FEDABAA89AF3031F4AEA9A43618F429
:10235E00EEA9EB5FEEABAA89A03131F4AFA9A4369A
:10236E0018F4EFA9EB5FEFABAA89A13131F4A9A95B
:10237E00A83C18F4E9A9EB5FE9ABAA89A23131F4C4
:10238E00AAA9A83C18F4EAA9EB5FEAABAA89A33183
:10239E0031F4ABA9A83C18F4EBA9EB5FEBABAA891F
:1023AE00A43169F4A0916903B0916A03A835E2E003
:1023BE00BE0728F40E94B5327E960E941933AA8970
:1023CE00A531D1F40E943336E0EFF0E00E945D3E7D
:1023DE000E943C36E8E6F1E00E945D3E0E944736E0
:1023EE00E0EEF1E00E945D3EE021E12929F0EF8D63
:1023FE00F8A13196EF8FF8A3AA89A63149F4A091DE
:10240E003303A13028F4E0913303EF5FE0933303FD
:10241E00AA89A73149F4A0913503A23328F4E0919B
:10242E003503EF5FE0933503AA89A83149F4A091F3
:10243E003403A13028F4E0913403EF5FE0933403CA
:10244E00AA89A931E1F4AF89B88DE9E1F0E00E94E3
:10245E0052360E94AD3329F0EF89F88D3196EF8B0D
:10246E00F88FAF89B88DE2E3F0E00E9452360E94F9
:10247E00BA3429F0EF89F88D3196EF8BF88FAA894F
:10248E00AA3159F40E945936A03BE4E0BE0728F465
:10249E000E940A3631960E945E36AA89AB3191F4BB
:1024AE000E940D32A73EE3E0BE07E0E08E07E0E0BB
:1024BE009E0740F40E94D531EF5FFF4F6F4F7F4F65
:1024CE000E941033AA89AC3161F4A0E023FCA1E094
:1024DE00A13038F4E0E023FCE1E0EF5F0E94D33F4F
:1024EE0023F8AA89AD3169F40E948531AE3DE3E04F
:1024FE00BE0738F40E9466313A96E0936103F0937A
:10250E006203AA89AE3169F40E948F31A835E2E0E8
:10251E00BE0738F40E9472313A96E0936D03F09341
:10252E006E03AA89AF3149F4A0910603AA3028F4AC
:10253E00E0910603EF5FE0930603AA89A03249F407
:10254E00A0910803AC3028F4E0910803EF5FE0930C
:10255E000803AA89A13249F4A0910903AC3028F4EA
:10256E00E0910903EF5FE0930903AA89A23249F4CF
:10257E00A0910A03AC3028F4E0910A03EF5FE093D8
:10258E000A03AA89A33249F4A0910B03AC3028F4B4
:10259E00E0910B03EF5FE0930B03AA89A43249F499
:1025AE00A0910C03AC3028F4E0910C03EF5FE093A4
:1025BE000C03AA89A53249F4A0912903A33028F46B
:1025CE00E0912903EF5FE0932903AA89A63249F42B
:1025DE00A0912A03A13028F4E0912A03EF5FE09343
:1025EE002A03AA89A73249F4A0912B03A23028F41A
:1025FE00E0912B03EF5FE0932B03AA89A83249F4F5
:10260E00A0912C03A13028F4E0912C03EF5FE0930E
:10261E002C03AA89A93249F4A0912D03A23028F4E3
:10262E00E0912D03EF5FE0932D03AA89AA3249F4BE
:10263E00A0912E03A33028F4E0912E03EF5FE093D8
:10264E002E03AA89AB3249F4A0912F03A13028F4AE
:10265E00E0912F03EF5FE0932F03AA89AC3249F488
:10266E00A0913003A13028F4E0913003EF5FE093A6
:10267E003003AA89AD3291F40E948932AF39E6E86F
:10268E00BE07E1E08E07E0E09E0740F40E94713243
:10269E00E65FFF4F6F4F7F4F0E947A32AA89AE32AC
:1026AE0059F40E947736A031E7E2BE0728F40E9463
:1026BE00F1313A960E94F631AA89AF3261F4A0E068
:1026CE0036FCA1E0A13038F4E0E036FCE1E0EF5F4B
:1026DE000E94D33F36F8AA89A03349F4A091100383
:1026EE00A13028F4E0911003EF5FE0931003AA8964
:1026FE00A13331F4ACA5A33018F4ECA5EF5FECA731
:10270E00AA89A23359F4AB8DBC8DA435E2E0BE0785
:10271E0028F4EB8DFC8D3196EB8FFC8FAA89A333B9
:10272E0049F4A0911503A43628F4E0911503EF5F48
:10273E00E0931503AA89A43341F40E947C36A23893
:10274E0020F40E948336EF5FEC93AA89A53349F4F7
:10275E00A0914E03A13028F4E0914E03EF5FE09379
:10276E004E03AA89AC3549F4A0910503AA3F28F47B
:10277E00E0910503EB5FE0930503AA89AD3531F4D3
:10278E00ACADA93018F4ECADEF5FECAFAA89AE3565
:10279E0049F4A0914903A93028F4E0914903EF5F71
:1027AE00E0934903AA89AF3559F4ABA1BCA1A83B6C
:1027BE00EBE0BE0728F4EBA1FCA13196EBA3FCA342
:1027CE00AA89A03659F4A98DBA8DA83EE3E0BE07BA
:1027DE0028F4E98DFA8D3A96E98FFA8FAA89A136F7
:1027EE0049F4A0912503AC3328F4E0912503EF5F63
:1027FE00E0932503AA89A23691F40E94E835A081C0
:10280E00AA3F21F40E948A36EB5FEC930E94E835D2
:10281E00A081AA3F20F40E948A36E65FEC930E94C4
:10282E0091360E94573EE02149F0A0911C03AA3F29
:10283E0028F4E0911C03E65FE0931C030E9491369E
:10284E000E94633EE02149F0A0911D03AA3F28F4A7
:10285E00E0911D03E65FE0931D03EAE0EB1510F433
:10286E00E894F2F8AB2DEAE00E94353E0E2EA0E081
:10287E00F2FCA1E00E9430350E940F3609F414C319
:10288E006894F2F8AA89A13049F4A0911703A130F7
:10289E0028F0E0911703E150E0931703AA89A230C4
:1028AE0031F4AFA1A63018F0EFA1E150EFA3AA8941
:1028BE00A33049F4A0911803AD3328F0E09118032A
:1028CE00E1500E942036AA89A43049F4A0911A033F
:1028DE00A53128F0E0911A03E150E0931A03AA897A
:1028EE00A53031F4A9ADA13018F0E9ADE150E9AF52
:1028FE00AA89A63031F4AAADA13018F0EAADE150A4
:10290E00EAAFAA89A73031F4ABADA13018F0EBAD28
:10291E00E150EBAFAA89A83049F4A0911B03A13076
:10292E0028F0E0911B03E150E0931B03AA89A93024
:10293E0049F4A0914103A13028F0E0914103E15008
:10294E00E0934103AA89AA3049F4A0914203A13031
:10295E0028F0E0914203E150E0934203AA89AB30A4
:10296E0049F4A0914303A13028F0E0914303E150D4
:10297E00E0934303AA89AC3049F4A0910E03A93128
:10298E0028F0E0910E03EC50E0930E03AA89AD30CF
:10299E0069F4A0915903B0915A03A538E3E0BE073C
:1029AE0028F00E94723331970E94FB32AA89AE3012
:1029BE0031F4ADA9A63018F0EDA9E550EDABAA891A
:1029CE00AF3031F4AEA9A63018F0EEA9E550EEAB5B
:1029DE00AA89A03131F4AFA9A63018F0EFA9E550BD
:1029EE00EFABAA89A13131F4A9A9A13018F0E9A958
:1029FE00E550E9ABAA89A23131F4AAA9A13018F0A9
:102A0E00EAA9E550EAABAA89A33131F4ABA9A1300A
:102A1E0018F0EBA9E550EBABAA89A43161F4A091B3
:102A2E006903B0916A030E94BF3F28F40E94B53239
:102A3E007E970E941933AA89A531D1F40E943336AC
:102A4E00EBECF0E00E94633E0E943C36E2E2F1E0E5
:102A5E000E94633E0E944736E9E7F1E00E94633E22
:102A6E00E021E12929F0EF8DF8A13197EF8FF8A33E
:102A7E00AA89A63149F4A0913303A13028F0E09140
:102A8E003303E150E0933303AA89A73149F4A091AF
:102A9E003503A23028F0E0913503E150E093350381
:102AAE00AA89A83149F4A0913403A13028F0E0910D
:102ABE003403E150E0933403AA89A93149F4AF8974
:102ACE00B88D129728F0EF89F88D3197EF8BF88F2C
:102ADE00AA89AA3159F40E945936A73DE1E0BE07F2
:102AEE0028F00E940A3631970E945E36AA89AB31D1
:102AFE0091F40E940D32AB30E0E0BE07E0E08E07AD
:102B0E00E0E09E0740F00E94D531E150F040604079
:102B1E0070400E941033AA89AC3159F4A0E023FC16
:102B2E00A1E0A13030F0A0E023FCA1E00E94973696
:102B3E0023F8AA89AD3161F40E9485310E94BF3F0E
:102B4E0038F40E9466313197E0936103F09362038B
:102B5E00AA89AE3161F40E948F310E94BF3F38F4D2
:102B6E000E9472313197E0936D03F0936E03AA8940
:102B7E00AF3149F4A0910603A23028F0E09106038C
:102B8E00E150E0930603AA89A03249F4A09108030C
:102B9E00A23028F0E0910803E150E0930803AA89DF
:102BAE00A13249F4A0910903A13028F0E091090364
:102BBE00E150E0930903AA89A23249F4A0910A03D5
:102BCE00A13028F0E0910A03E150E0930A03AA89AC
:102BDE00A33249F4A0910B03A13028F0E0910B032E
:102BEE00E150E0930B03AA89A43249F4A0910C039F
:102BFE00A13028F0E0910C03E150E0930C03AA8978
:102C0E00A53249F4A0912903A13028F0E0912903BF
:102C1E00E150E0932903AA89A63249F4A0912A0330
:102C2E00A13028F0E0912A03E150E0932A03AA890B
:102C3E00A73249F4A0912B03A13028F0E0912B0389
:102C4E00E150E0932B03AA89A83249F4A0912C03FA
:102C5E00A13028F0E0912C03E150E0932C03AA89D7
:102C6E00A93249F4A0912D03A13028F0E0912D0353
:102C7E00E150E0932D03AA89AA3249F4A0912E03C4
:102C8E00A13028F0E0912E03E150E0932E03AA89A3
:102C9E00AB3249F4A0912F03A13028F0E0912F031D
:102CAE00E150E0932F03AA89AC3249F4A09130038E
:102CBE00A13028F0E0913003E150E0933003AA896F
:102CCE00AD3269F40E9489320E94C33F40F40E94E3
:102CDE007132E150F040604070400E947A32AA8911
:102CEE00AE3251F40E9477360E94BF3F28F40E9404
:102CFE00F13131970E94F631AA89AF3259F4A0E032
:102D0E0036FCA1E0A13030F0A0E036FCA1E00E943C
:102D1E00973636F8AA89A03349F4A0911003A13052
:102D2E0028F0E0911003E150E0931003AA89A1333B
:102D3E0031F4ACA5A13018F0ECA5E150ECA7AA89AE
:102D4E00A23359F4AB8DBC8DA53FE0E0BE0728F051
:102D5E00EB8DFC8D3197EB8FFC8FAA89A33349F451
:102D6E00A0911503A23028F0E0911503E150E093F5
:102D7E001503AA89A43341F40E947C36A53120F0B4
:102D8E000E948336E150EC93AA89A53349F4A091B1
:102D9E004E03A13028F0E0914E03E150E0934E0334
:102DAE00AA89AC3549F4A0910503A13028F0E09131
:102DBE000503E550E0930503AA89AD3531F4ACADBA
:102DCE00A13018F0ECADE150ECAFAA89AE3549F464
:102DDE00A0914903A13028F0E0914903E150E0931E
:102DEE004903AA89AF3559F4ABA1BCA1A13DE7E0D7
:102DFE00BE0728F0EBA1FCA13197EBA3FCA3AA8997
:102E0E00A03659F4A98DBA8DA536E0E0BE0728F09C
:102E1E00E98DFA8D3A97E98FFA8FAA89A13649F48E
:102E2E00A0912503A13028F0E0912503E150E09315
:102E3E002503AA89A236D1F40E94E835BF01A081EC
:102E4E000E949632FB01A081EFEF0E94353EE021F9
:102E5E0021F00E948A36EA50EC930E94E835A08158
:102E6E00AF3F21F40E948A36E550EC930E949136D2
:102E7E000E94573EE02149F0A0911C03A13028F09A
:102E8E00E0911C03EA50E0931C030E9491360E94CD
:102E9E00633EE02149F0A0911D03A13028F0E0919E
:102EAE001D03EA50E0931D0323FC6EC00E949E3664
:102EBE00ACA50E94F633ACA5E3E00E94173EE029D4
:102ECE0041F00E949E360E944D350E9407330E94AB
:102EDE00A6360E944D35E0E0F0E06EEF72E40E94FF
:102EEE00A23D09F008F40AC00E94A936A0E0B0E0A5
:102EFE0080E893E40E94B83C0E94A636E091480315
:102F0E00F0E0E0939F03F093A0030E94AC36A0384C
:102F1E00E0E0BE0754F0E0919F03F091A003E05073
:102F2E00F140E0939F03F093A003ACA5A33001F111
:102F3E000E944D350E94C33F3CF40E94B1360E9460
:102F4E00BF3C0E94B73613C0AB81AA233AF40E944D
:102F5E00B1360E94B83C0E94B73609C0E0E0E0935B
:102F6E00DB03E093DC03E093DD03E093DE0304C0B8
:102F7E000E94A9360E94B7360E94C036ADE8B3E073
:102F8E000E9416320E94C23623FE43C0EB89FC8992
:102F9E000E945E35EC83FD836E837F83AC81BD81A1
:102FAE008E819F81E0E0F0E060E874E40E945D3D78
:102FBE00A0E0B0E48CE995E40E940F3DDF01CB0167
:102FCE00EBA1FCA10E9450350E94C731DF01CB015D
:102FDE00E3E3F3E365E872E40E945D3D0E94A636EA
:102FEE00A0910F03A13018F4E0E00E946D3F0E9403
:102FFE00A9360E94B736E0910603A0910703AE17DB
:10300E0040F00E94C036ADE8B3E00E9416320E9436
:10301E00C236A0E0F0FCA1E00E94C636E0910603A5
:10302E00A09107030E94303EE02109F446C0E091D2
:10303E002C03E030F1F4AD89BE89E0E0F4E00E94AB
:10304E00CB36A3E9B3E00E941632E0919B03F091D8
:10305E009C030E94DD36A5E9B3E00E941632E09192
:10306E009D03F0919E030E94DD36A7E9B3E00E9416
:10307E001632A0912C03A130E9F4AB89BC89E2E0B1
:10308E00F0E00E94DC3E3597E0939303F0939403B7
:10309E00E0919B03F0919C033597E0939503F09399
:1030AE009603E0919D03F0919E033597E09397036D
:1030BE00F0939803E0E0E0930703F0916F03E0E0F4
:1030CE00DF01E0913903F0E0EA0FFB1FABEBB3E059
:1030DE000E946B310E94E436A0E0B0E080E192E401
:1030EE000E945D3D7F936F93FF93EF930E9459363D
:1030FE000E94ED36AF91BF918F919F910E945035F6
:10310E000E940F3DE093BB03F093BC036093BD039D
:10311E007093BE030E94F236E0E0F0E060E87FE3D9
:10312E000E94C83D0E2E0E94F236E0E0F0E068EC00
:10313E0072E40E94C23D0E220E94F236E0E0F0E8F8
:10314E006BE375E40E94713EE02109F10E94E436C2
:10315E00A0E0B0E080E09FE30E94BF3CABEAB3E0AA
:10316E000E944E3C0E94593F0E94E436E093BF03FA
:10317E00F093C0036093C1037093C2030E94F236B2
:10318E000E949232ABE5B3E00E949D3115C0E0E0A3
:10319E00E093AB03E093AC03E093AD03E093AE0397
:1031AE00E093BF03E093C003E093C103E093C20337
:1031BE00E0935B03E0935C030E9422320E94BD31D8
:1031CE000E94C83DEF930E94D5310E94DE310E94CD
:1031DE00C83DAF91EA23C1F10E94B431E0E0F0E0C6
:1031EE0068EC72E40E945D3D0E940D320E94723FB7
:1031FE000E94C7310E94FB36A091B703B091B8036D
:10320E008091B9039091BA03E0E0F0E064E172E4DA
:10321E000E940F3DDF01CB010E9432320E945D3DC4
:10322E00A0E0B0E080E291E40E940F3D0E94FB36E8
:10323E00E091B703F091B8036091B9037091BA03AE
:10324E00DE0150960E9416320E94E733A0912303AE
:10325E00EDEF0E94353E0E220E949B34E02129F0B4
:10326E00E0912303EF5FE0932303A62D0E94DA354E
:10327E00A0912303EFEF0E94353E0E220E949B3455
:10328E00E02129F0E894F0F8E0E0E0932303A09128
:10329E002303EEE10E94173E0E2E0E949B34E02186
:1032AE0019F0E1E0E0932603E0912503E03019F4F4
:1032BE00E0E0E09326030E9404370E94A735A09118
:1032CE002603E0E00E943A3EE02119F0E1E0E093AF
:1032DE002603A0912603AC3321F4E8ECF0E0EDA335
:1032EE00FEA3A0910503A13028F0E0910503F0E0C4
:1032FE000E94C233A09130030E94F6330E9496358D
:10330E00E02159F1EBA5EF5FEBA7F0E03196BF019D
:10331E00ADA1BEA10E94ED36E617F70790F40E940C
:10332E0009370E94793E0E2E0E941237E4EAF1E030
:10333E0060E070E00E94693EE02919F0E0E0EDA344
:10334E00EEA3ADA1BEA10E94ED36ABA5B0E0EA178B
:10335E00FB0710F4E0E0EBA702C0E0E0EBA70E9451
:10336E0096350E2E0E9409370E94893E0E22AB8D95
:10337E00BC8DE4EAF1E00E94453EE02151F0ADA1A2
:10338E00BEA1A639E0E0BE0720F4E6E9F0E0EDA329
:10339E00FEA3ECA5E03009F094C04420B1F5E09115
:1033AE001403E03041F4E12FF0E034960E949433A0
:1033BE00EA0FFB1F03C00E9403343F96ADA1BEA1CE
:1033CE00EA0FFB1FBF01A0913103B0E0E7E00E94BE
:1033DE00EC3DE60FF71F0E941737AEE30E94473110
:1033EE00A4E00E944731E0911403E03011F4A12FC4
:1033FE0001C0ABE00E944731E09131030E941C37BF
:10340E000E942137ADA10E942737E1E0E41509F0B3
:10341E0058C04424A0911803B0E0E2E0F0E00E940E
:10342E00DC3EE0931903F0E0BC96DF01E091160359
:10343E00F0E0AE0FBF1FE0911703F0E0AE0FBF1F1D
:10344E00EFA10E943237AE0FBF1FE9ADF0E0AE0F15
:10345E00BF1FEAADF0E0AE0FBF1FEBADF0E0AE0F59
:10346E00BF1FE0911B030E943937F0E0AE0FBF1F64
:10347E00E0914303F0E0EA0FFB1F0E941737AEE323
:10348E000E944731ACE20E944437AFA10E944731FF
:10349E00A09119030E944E37A9AD0E944731AAADE3
:1034AE000E944731ABAD0E945437A09141030E9458
:1034BE004731A09142030E944731A09143030E94DD
:1034CE002737ACA5A13009F070C0E0913103EE0FA3
:1034DE00EE0FE0933103EF5FE0933103ADA1BEA198
:1034EE00A93CE0E0BE0720F0E8ECF0E0EDA3FEA37F
:1034FE00ADA1BEA1E5E00E94B93EEDA3FEA30E94E0
:10350E009433E5E00E94B93E0E94C233E09131034C
:10351E00AFE2EA27A0911A03AE27E1E0AE27E6E379
:10352E00AE27EEA1F070EA27ADA1BEA1AE27BF2750
:10353E00E0915003F070EA27FB270E949433AE27E8
:10354E00BF27E1E0F0E0AE27BF27E6E3F0E0AE27CD
:10355E00BF27EFA1F0E0AE27BF27E12FF0E0EA276B
:10356E00FB270E941737AFE20E944731A09131032B
:10357E000E944731A0E00E944E370E945A37AEA1FA
:10358E000E944731ADA10E944731E0915003AE2F0A
:10359E000E9421370E945A37A0E00E944731AFA106
:1035AE000E944731A12F0E946037ACA5A33009F0CD
:1035BE0092C0442009F047C0E0911403E03051F46A
:1035CE00E12FF0E03596DF01E0914403F0E0AE0F1D
:1035DE00BF1F05C0E0914403F0E07096DF01E0915B
:1035EE004503F0E0AE0FBF1FE0914603F0E0EA0F97
:1035FE00FB1F0E949433EA0FFB1FADA1BEA1EA0F81
:10360E00FB1F0E941737AEE60E944731A5E00E94CD
:10361E004731E0911403E03011F4A12F01C0ABE06B
:10362E000E944731A09144030E944731A091450367
:10363E000E944731A09146030E942137ADA10E94FE
:10364E0066370E946037E1E0E41509F044C0442477
:10365E00E0911603F0E0BD96DF01E09117030E94A2
:10366E0039370E943237AE0FBF1FD296E0911B033F
:10367E00F0E0AE0FBF1FE0911503F0E0EA0FFB1F65
:10368E007E2F8F2FAF89B88DEAE00E94B93EE70FEB
:10369E00F81F0E941737AEE60E944731ADE20E9436
:1036AE004437A09142030E944731A09141030E94EA
:1036BE004E37A2E30E9466370E945437EF89AAE084
:1036CE00EA9FF001AE2F0E944731A09115030E9490
:1036DE0066370E9460370E946D370E949B32FF272B
:1036EE00662777270E94C93F34F4E091AB03A6E327
:1036FE00B0E00E94A83F0E9472370E944D35FF270E
:10370E00662777270E94853C0E94A23D09F008F4A7
:10371E0008C00E94A936A7E3B0E00E944C3C0E946C
:10372E00A83F0E9477370E94AC36F0E0EA17FB07FD
:10373E0034F4E0919F03A8E3B0E00E94A83F0E94FA
:10374E007C370E9481370E940D3E0E94813E0E2ED4
:10375E000E948137E8ECF0E060E070E00E94893E64
:10376E00E02131F0EC85FD85A1E5B0E00E94A03F9F
:10377E000E9486370E9481370E940D3E0E94C93FEB
:10378E0034F4EC85FD85A3E5B0E00E94A03F0E94D5
:10379E008B37A0919303B0919403EA17FB0744F47F
:1037AE00E0919303F0919403A7E5B0E00E94A03F4F
:1037BE000E949037A0919503B09196030E94513EBE
:1037CE000E94CC340E94A434E02141F0E091950394
:1037DE00F0919603A9E5B0E00E94A03F0E949537B4
:1037EE00A0919703B09198030E94513E0E94CC3451
:1037FE000E94A434E02141F0E0919703F0919803E8
:10380E00ABE5B0E00E94A03F0E941E330E94C23181
:10381E00AE1BBF0BA436E0E0BE0710F00E94D13500
:10382E00EC85FD856E857F850E944D350E94853C19
:10383E000E940F3DA1EAB3E00E9416320E949A3711
:10384E000E949F37E093A103F093A2030E94A43736
:10385E000E949A37EA17FB0744F4E091A103F09116
:10386E00A203A5E5B0E00E94A03F033608F0E1C731
:10387E000E9404360081A0913703A13048F420FC49
:10388E0007C0A0E0F799A1E0EA2FE295E07F19C00A
:10389E00A0E0F799A1E0EA2FE295E07F0E2EA0E0DE
:1038AE00F399A1E0EA2FEE0FEE0F0E0EA0E0F499C1
:1038BE00A1E0EA2FEE0FA02DAE0FE0E0F599E1E0CA
:1038CE00EA0FEDAF0E944D35EDECFCEC6CEC7DEBB0
:1038DE000E94A23D18F4EDADE05AEDAFEAE00E9471
:1038EE00A937EAE0DE01AF5ABF4FEC930E94AE3724
:1038FE000E94B437EAE00E94B937EAE00E94BE3770
:10390E00EAE00E94C3370E94C837E89435F8A0E079
:10391E0031FCA1E00E94F633A0E032FCA1E0E1E030
:10392E000E94173E0E2AA0E034FCA1E0E1E00E94C6
:10393E00173EE02911F020FA01C0E894F5F8E09165
:10394E002E03E03021F40E94EA370E94FA37A0914C
:10395E002E03A13081F4A0E022FCA1E0EA2FEE0FAD
:10396E00E75F0E2EA0E022FCA1E0EA2FEE0FEE0F95
:10397E00E00D0E940938A0912E03A23099F40E9406
:10398E00EA37A0E022FCA1E0EA2F0E9419380E0EC1
:10399E00A0E022FCA1E0EA2FE295E07FEE0F0E0EF2
:1039AE000E94FA37A0912E03A33031F4E0E022FCFE
:1039BE00E1E0E85F0E940938A0910E03A83109F0FA
:1039CE0041C00E941E38A23DE0E0BE07E0E08E0737
:1039DE00E0E09E071CF0E1E0E09301030E948137D6
:1039EE00A83FE0E0BE07E0E08E07E0E09E071CF097
:1039FE00E3E0E09301030E948137AF3FE0E0BE07B2
:103A0E00E0E08E07E0E09E071CF0E7E0E0930103A4
:103A1E000E948137A430E1E0BE07E0E08E07E0E0CF
:103A2E009E071CF0EFE0E09301030E948137AE3059
:103A3E00E1E0BE07E0E08E07E0E09E071CF0EFE15C
:103A4E00E0930103A0910E03A43209F041C00E943D
:103A5E001E38A633E1E0BE07E0E08E07E0E09E07E9
:103A6E001CF0E1E0E09301030E948137AA34E1E00B
:103A7E00BE07E0E08E07E0E09E071CF0E3E0E09377
:103A8E0001030E948137AE35E1E0BE07E0E08E070C
:103A9E00E0E09E071CF0E7E0E09301030E9481370F
:103AAE00A836E1E0BE07E0E08E07E0E09E071CF0DE
:103ABE00EFE0E09301030E948137AC37E1E0BE07EF
:103ACE00E0E08E07E0E09E071CF0EFE1E0930103DB
:103ADE00A0910E03A03309F041C00E941E38A638F3
:103AEE00E1E0BE07E0E08E07E0E09E071CF0E1E0BB
:103AFE00E09301030E948137AC3CE1E0BE07E0E0B9
:103B0E008E07E0E09E071CF0E3E0E09301030E94C5
:103B1E008137A63DE1E0BE07E0E08E07E0E09E07BC
:103B2E001CF0E7E0E09301030E948137A03EE1E044
:103B3E00BE07E0E08E07E0E09E071CF0EFE0E093AA
:103B4E0001030E948137AF3EE1E0BE07E0E08E0741
:103B5E00E0E09E071CF0EFE1E0930103A091140357
:103B6E00A13081F4A0E020FCA1E0EA2F0E941938D8
:103B7E000E2EA0E020FCA1E0EA2FE295E07FEE0FF2
:103B8E00E00D4E0FA0910203A431F0F40E949B327F
:103B9E000E9424386CF0FE01E15BFF4F3396FF93D9
:103BAE00EF930E942C380E943238AF91BF91EC9364
:103BBE000E943D38FF93EF930E942C380E94203FC5
:103BCE00AF91BF91EC930DC020FE05C0E0E40E94C2
:103BDE004238E0E402C00E94AE37DE01AD5ABF4F5C
:103BEE00EC93AAA5A13090F0EAA5E150EAA7E8E788
:103BFE000E944238E0911403E03029F4FE01E15BAB
:103C0E00FF4F148303C0E0E50E94B437A9A5A1308D
:103C1E0058F0E9A5E150E9A7E8E30E9442380E9476
:103C2E003D38A0913203A083A8A5A13048F0E8A5A5
:103C3E00E150E8A7E9E30E944238E0E50E94B4377C
:103C4E00E0911103E03019F54058A0918E03AA239C
:103C5E0092F4E0E40E94A937A0918D03B0918E03F7
:103C6E00AD39EFEFBE0714F4689435F80E9447386B
:103C7E000E944F3802C0E89435F80E9454381A97C3
:103C8E0024F00E9459380E9460380E946838A09132
:103C9E001103A13009F045C0EDADE85FEDAF0E9414
:103CAE007538FF2392F4E0E40E94A9370E9475381C
:103CBE00E73FAFEFFA0714F4689401C0E89435F8C3
:103CCE000E9475380E94D83D04C0E89435F80E94D1
:103CDE007538E0938F03F09390030E9454381A972F
:103CEE0024F00E9459380E9460380E9468380E9461
:103CFE007538BF01DF01E3E6F0E00E94513E0E2E63
:103D0E00DB01EDE9FFEF0E944B3EE02951F0E89414
:103D1E0035F8E0E40E94A937E0E4DE01AF5ABF4F68
:103D2E00EC930E948138FF93EF930E9481370E949B
:103D3E0086380E943238AF91BF910E948B383696EA
:103D4E00FF93EF930E9490380E943238AF91BF914B
:103D5E000E948B383796FF93EF930E9490380E9403
:103D6E00203FAF91BF91EC930E948137A639E0E0DE
:103D7E00BE07E0E08E07E0E09E0764F4E0E40E94F8
:103D8E00B937E0E40E94BE37E0E40E94C337E0E0BA
:103D9E00E0930103013009F05BC00E9496380E9447
:103DAE009E38A83EE3E0BE07B8F0505E0E94A338EE
:103DBE000E94A9380E948B383E96BF010E949E3801
:103DCE000E94B4380E948B383F96BF010E949E38E5
:103DDE000E94ED36DF011BC050560E949E38A4365D
:103DEE00E0E0BE0728F00E94A3380E94B438EC939E
:103DFE000E94BF38BF010E949E380E94ED360E947D
:103E0E00C4380E948B383F96BF010E949E38EAE06C
:103E1E00F0E00E94CB38A0910003AA3010F00E946F
:103E2E00D0380E94D638A09100030E94DC380E9440
:103E3E008B383A96BF01AC2DB0E00E949F370E949E
:103E4E0060380E94E338BF01AC2D0E94DC38EC9341
:103E5E00023009F06DC0505C0E948932A03AE6E84B
:103E6E00BE07E1E08E07E0E09E0778F00E94E8389A
:103E7E00FF93EF930E948932E0EAF6E861E070E08A
:103E8E000E94ED38AF91BF91EC930E9489320E944F
:103E9E00F83878F00E94E338FF93EF930E9489324E
:103EAE00E0E1F7E260E070E00E94ED38AF91BF9183
:103EBE00EC930E9489320E94003968F00E94083902
:103ECE00FF93EF930E9489320E9496340E94ED3840
:103EDE00AF91BF91EC930E9489320E940D3968F028
:103EEE000E941539FF93EF930E9489320E94863803
:103EFE000E94ED38AF91BF91EC930E9489320E94DF
:103F0E00243858F00E94BF38FF93EF930E941A395D
:103F1E000E94ED38AF91BF91EC930E942039FF9330
:103F2E00EF930E941A390E941C3FAF91BF91EC9300
:103F3E00033009F0BDC0E7E70E9425390E942F39F2
:103F4E000E94F8387CF00E94E338FF93EF930E94B2
:103F5E002F39E0E1F7E260E070E00E943238AF9175
:103F6E00BF91EC930E942F390E9400396CF00E9491
:103F7E000839FF93EF930E942F390E9496340E94C6
:103F8E003238AF91BF91EC930E942F390E940D39B8
:103F9E005CF00E941539FF93EF930E942F390E9417
:103FAE003839AF91BF91EC930E942F390E9424387B
:103FBE005CF00E94BF38FF93EF930E943A390E9443
:103FCE003238AF91BF91EC93A091B203AA235AF06D
:103FDE000E942039FF93EF930E943A390E94203FAE
:103FEE00AF91BF91EC93A091B203AA2372F40E94F9
:103FFE002039FF93EF930E9440390E94203FAF91EA
:10400E00BF91EC93E0E40E9451390E942F39A73FF3
:10401E00EFEFBE07EFEF8E07EFEF9E076CF40E94F7
:10402E00BF38FF93EF930E9440390E943238AF9110
:10403E00BF91EC930E9456390E942F39AD39EFEFA4
:10404E00BE07EFEF8E07EFEF9E076CF40E94153957
:10405E00FF93EF930E945C390E943839AF91BF9164
:10406E00EC930E9469390E942F39A931ECEFBE07FB
:10407E00EFEF8E07EFEF9E077CF40E940839FF9357
:10408E00EF930E945C390E9496340E943238AF91B1
:10409E00BF91EC930E946F390E942F39A13FE8ED3A
:1040AE00BE07EFEF8E07EFEF9E0714F40E947539EF
:1040BE00A02F0E94CD33A02FE9E00E94173EE029E9
:1040CE0009F480C05058093011F40E94D038EEE344
:1040DE000E9425390E948039A031E7E2BE074CF0DC
:1040EE000E94E338BF010E948039E0E1F7E20E94AE
:1040FE0085390E948039A83EE3E0BE073CF00E945D
:10410E000839BF010E9480390E9488390E94803987
:10411E00A436E0E0BE073CF00E941539BF010E94B4
:10412E0080390E948B39A0918A03AA2382F00E94C3
:10413E00BF38BF010E9480390E949F370E946038AD
:10414E000E942039BF010E9480390E948E39A091B1
:10415E008A03AA238AF40E94BF380E949539DF0190
:10416E000E949F370E9460380E9420390E94953924
:10417E000E9460380E9456390E948039AD39EFEFA7
:10418E00BE074CF40E9415390E949539DF010E943A
:10419E008B390E9469390E948039A931ECEFBE0734
:1041AE004CF40E9408390E949539DF010E9488392B
:1041BE000E946F390E948039A13FE8EDBE0714F4CA
:1041CE000E947539A02F0E949D39A02FEAE00E940F
:1041DE00173EE029C1F150580A3011F40E94D03830
:1041EE00EEE30E9425390E94A239A091E203AA2390
:1041FE0012F40E9456390E942232E0E0F0E066ECA2
:10420E0072EC0E94A23D10F40E9469390E94A839F6
:10421E00A436E0E0BE073CF00E941539BF010E94B3
:10422E00A8390E948B390E94BF38BF010E94A8395D
:10423E000E949F370E9460380E942039BF010E9461
:10424E00A8390E948E390630A1F55058E0E00E9440
:10425E00AD39E5E00E94B239E8E70E94B739A88986
:10426E00B989A83EE3E0BE073CF00E940839BF01C1
:10427E00A889B9890E948839A889B989A436E0E04D
:10428E00BE073CF00E941539BF01A889B9890E946A
:10429E008B390E94BF38BF01A889B9890E949F3708
:1042AE000E9460380E942039BF01A889B9890E94F6
:1042BE008E39073009F084C0ADA1BEA10E94BF3F68
:1042CE0030F5ECE00E94AD390E94BC39E436A0E036
:1042DE00FA0740F00E94E838BF01ADA1BEA10E94CE
:1042EE00C139EC930E94BC393A9740F00E94E338F2
:1042FE00BF01ADA1BEA10E94C639EC930E94083940
:10430E00BF010E94BC390E94C438EC9359C0A091E1
:10431E0042030E94C636A0914203E2E00E94173E7D
:10432E00E02929F1EBE00E94AD390E94CB39E43649
:10433E00A0E0FA0740F00E94E838BF01AD8DBE8DB7
:10434E000E94C139EC930E94CB393A9740F00E94FB
:10435E00E338BF01AD8DBE8D0E94C639EC930E942D
:10436E000839BF010E94CB390E94C438EC93A0914A
:10437E0042030E94F633A0914203E3E00E94173EEF
:10438E00E029F1F0EBE00E94AD39AD8DBE8DA43683
:10439E00E0E0BE0740F00E94E838BF01AD8DBE8D53
:1043AE000E94B438EC930E94E338BF01AD8DBE8DF0
:1043BE000E94ED360E94C438EC93E7E70E94D03994
:1043CE00083009F07EC00E949638A0918503B09106
:1043DE008603A135EBEFBE0734F4E1E5FBEFE09386
:1043EE008503F0938603A0918503B0918603A03BCD
:1043FE00E4E0BE0734F0EFEAF4E0E0938503F093D7
:10440E008603A0918603AA234AF40E946939E0919B
:10441E008503F09186030E94D83D04C0E091850388
:10442E00F0918603E0938703F0938803A0918703AE
:10443E00B0918803ECE3F0E00E94DC3EE09363036E
:10444E00F09364030E94D539ECE30E94B93EA0912B
:10445E008703B0918803AE1BBF0BA0936503B09387
:10446E00660324FE25C00E94D5391A9710F00E94CB
:10447E00D0380E94D6380E94D539EAE0F0E00E948A
:10448E000B3FDB010E948B383A96BF01A09165036A
:10449E00B09166030E94ED360E94C4380E948B389C
:1044AE003B96BF01A0916503B09166030E94DA3975
:1044BE00E3E70E94DD39E8E30E945139E4E50E940A
:1044CE00E2390B30A1F55054E9E30E94B239E8E32A
:1044DE000E94B7390E947736A83EE3E0BE0740F04F
:1044EE000E940839BF010E9477360E94A938EC93CA
:1044FE000E947736A436E0E0BE0740F00E941539E0
:10450E00BF010E9477360E94B438EC930E94BF38E8
:10451E00BF010E9477360E94ED360E94C4380E9479
:10452E008B383F96BF010E9477360E94DA390C30E5
:10453E0009F074C00E94D038EEE30E94AD390E949B
:10454E009A37E0E0F0E00E94E739E6EFFFEF0E94D5
:10455E00513EE02119F0E0E40E9451390E949A3751
:10456E00E7EFFFEF0E94E739ECE9FFEF0E94513EC3
:10457E00E02111F00E9456390E949A37EDE9FFEFC3
:10458E000E94E739E8E1FCEF0E94513EE02111F074
:10459E000E9469390E949A37A931ECEFBE0714F4D4
:1045AE000E946F39A091A203AA2352F4E091A103B5
:1045BE00F091A2030E94D83DE093A103F093A203D1
:1045CE000E949A37A83EE3E0BE073CF00E940839ED
:1045DE00BF010E949A370E9488390E949A37A436EA
:1045EE00E0E0BE073CF00E941539BF010E949A37E9
:1045FE000E948B390E949A371A974CF00E94BF384E
:10460E00BF010E949A370E949F370E9460380E9415
:10461E002039BF010E949A370E948E39AFA50E94A1
:10462E009632AEA5E0E00E943A3EE02909F4AFC012
:10463E005F77E0913803E170EE0F4E23E09138037F
:10464E00E6950E94EB390E2EE0913803E695E6953D
:10465E00E170AE2FE0E0F5FCE1E0EA2BEE0FEE0F9D
:10466E00E00D4E0F0E94C837AEA50E949632AFA540
:10467E00E0E00E943A3EE02159F1AEA5A13029F4C6
:10468E000E94F039ECE00E94D039AEA5A23029F498
:10469E000E94F039EDE00E94D039AEA5A33029F486
:1046AE000E94F039EBE00E94D0390E94F33929F0D4
:1046BE000E94F039ECE00E94D0390E94D2330E9461
:1046CE00FD3929F00E94F039EBE00E94D0392AC062
:1046DE00AEA5A13029F40E94033AECE00E94E23923
:1046EE00AEA5A23029F40E94033AEDE00E94E23911
:1046FE00AEA5A33029F40E94033AEBE00E94E23902
:10470E000E94F33929F00E94033AECE00E94E2394C
:10471E000E94D2330E94FD3929F00E94033AEBE049
:10472E000E94E239AFA5A13029F40E94073AECE0CD
:10473E000E94E239AFA5A23029F40E94073AEDE0BB
:10474E000E94E239AFA5A33029F40E94073AEBE0AC
:10475E000E94E239AFA5E4E00E94173E0E94FD39A7
:10476E0029F00E94073AECE00E94E239AFA5E5E09D
:10477E000E94173E0E94FD3929F00E94073AEBE095
:10478E000E94E239E0911103E03009F44058E091C3
:10479E004A03A0919303B09194030E940B3A0E2EFC
:1047AE00A0914A030E940F3A31F0E0E00E94143AC1
:1047BE00E0E00E94183AA0919503B0919603E09123
:1047CE004B030E940B3A0E2EA0914B030E940F3A00
:1047DE0031F0E1E00E94143AE1E00E94183AA09113
:1047EE009703B0919803E0914C030E940B3A0E2E62
:1047FE00A0914C030E940F3AC1F0E2E00E94143ADD
:10480E00E2E00E94B239E0E00E94B739E9E70E9487
:10481E00D039E0E50E94DD39E0E50E945139E0E053
:10482E000E94E239E1E0E0933F03F29B02C04B7F2E
:10483E004F5F033611F00C940D2D31E0303140F402
:10484E000E94273AEAE0EC93E89435F83F5FF6CF02
:10485E00AA89EBE50E942F3AEAE50E94173EE0296D
:10486E0011F0E5E3EA8BAA89A63311F4ECE5EA8BA5
:10487E00EA89E03029F4E0911603F0E0E9A3FAA307
:10488E00AA89A13029F4E0911703F0E0E9A3FAA375
:10489E00AA89A23021F4EFA1F0E0E9A3FAA3AA8934
:1048AE00A33029F4E0911803F0E0E9A3FAA3AA8952
:1048BE00A43029F4E0911A03F0E0E9A3FAA3AA893F
:1048CE00A53021F4E9ADF0E0E9A3FAA3AA89A63058
:1048DE0021F4EAADF0E0E9A3FAA3AA89A73021F406
:1048EE00EBADF0E0E9A3FAA3AA89A83029F4E09190
:1048FE001B03F0E0E9A3FAA3AA89A93029F4E091F9
:10490E004103F0E0E9A3FAA3AA89AA3029F4E091C1
:10491E004203F0E0E9A3FAA3AA89AB3029F4E091AF
:10492E004303F0E0E9A3FAA3AA89AC3029F4E0919D
:10493E000E03F0E0E9A3FAA3AA89AD3021F40E9498
:10494E007233E9A3FAA3AA89AE3021F4EDA9F0E0FF
:10495E00E9A3FAA3AA89AF3021F4EEA9F0E0E9A306
:10496E00FAA3AA89A03121F4EFA9F0E0E9A3FAA3F2
:10497E00AA89A13121F4E9A9F0E0E9A3FAA3AA8951
:10498E00A23121F4EAA9F0E0E9A3FAA3AA89A3319E
:10499E0021F4EBA9F0E0E9A3FAA3AA89A43121F44A
:1049AE000E94B532E9A3FAA3AA89A53121F4EF8DAD
:1049BE00F8A1E9A3FAA3AA89A63129F4E091330359
:1049CE00F0E0E9A3FAA3AA89A73129F4E09135030F
:1049DE00F0E0E9A3FAA3AA89A83129F4E0913403FF
:1049EE00F0E0E9A3FAA3AA89A93121F4EF89F88DA1
:1049FE00E9A3FAA3AA89AA3121F40E940A36E9A3EF
:104A0E00FAA3AA89AB3131F4E0917B03F0917C03D8
:104A1E00E9A3FAA3AA89AC3131F4E0E023FCE1E08A
:104A2E00F0E0E9A3FAA3AA89AD3121F40E94663120
:104A3E00E9A3FAA3AA89AE3121F40E947231E9A347
:104A4E00FAA3AA89AF3129F4E0910603F0E0E9A3B5
:104A5E00FAA3AA89A03229F4E0910803F0E0E9A3B1
:104A6E00FAA3AA89A13229F4E0910903F0E0E9A39F
:104A7E00FAA3AA89A23229F4E0910A03F0E0E9A38D
:104A8E00FAA3AA89A33229F4E0910B03F0E0E9A37B
:104A9E00FAA3AA89A43229F4E0910C03F0E0E9A369
:104AAE00FAA3AA89A53229F4E0912903F0E0E9A33B
:104ABE00FAA3AA89A63229F4E0912A03F0E0E9A329
:104ACE00FAA3AA89A73229F4E0912B03F0E0E9A317
:104ADE00FAA3AA89A83229F4E0912C03F0E0E9A305
:104AEE00FAA3AA89A93229F4E0912D03F0E0E9A3F3
:104AFE00FAA3AA89AA3229F4E0912E03F0E0E9A3E1
:104B0E00FAA3AA89AB3229F4E0912F03F0E0E9A3CE
:104B1E00FAA3AA89AC3229F4E0913003F0E0E9A3BC
:104B2E00FAA3AA89AD3231F4E0917703F0917803BC
:104B3E00E9A3FAA3AA89AE3221F40E94F131E9A3C6
:104B4E00FAA3AA89AF3231F4E0E036FCE1E0F0E0FE
:104B5E00E9A3FAA3AA89A03329F4E0911003F0E0A7
:104B6E00E9A3FAA3AA89A13321F4ECA5F0E0E9A305
:104B7E00FAA3AA89A23321F4EB8DFC8DE9A3FAA343
:104B8E00AA89A33329F4E0911503F0E0E9A3FAA36F
:104B9E00AA89A43349F4E0912B03F0E0E65BFC4FC5
:104BAE00E081F0E0E9A3FAA3AA89A53329F4E09104
:104BBE004E03F0E0E9A3FAA3AA89AC3529F4E091FB
:104BCE000503F0E0E9A3FAA3AA89AD3521F4ECAD13
:104BDE00F0E0E9A3FAA3AA89AE3529F4E0914903DE
:104BEE00F0E0E9A3FAA3AA89AF3521F4EBA1FCA169
:104BFE00E9A3FAA3AA89A03621F4E98DFA8DE9A3D7
:104C0E00FAA3AA89A13629F4E0912503F0E0E9A3DD
:104C1E00FAA3AA89A23631F40E94E835E081F0E0C9
:104C2E00E9A3FAA30E9491360E94573EE02129F093
:104C3E00E0911C03F0E0E9A3FAA30E9491360E94D2
:104C4E00633EE02129F0E0911D03F0E0E9A3FAA311
:104C5E00AA890E94C636AA89E3E00E94343AE1E1AD
:104C6E000E94343AE2E10E94343AE3E10E94343A7F
:104C7E00E5E10E94343AEAE10E94343AEBE10E9407
:104C8E00343AEDE10E94343AEEE20E94173EE029FA
:104C9E001E2E0E94393A0E94453EE0211E2AAA8904
:104CAE00EEE50E94173E0E2EA0914903E2E00E940F
:104CBE003A3E0E22E5E00E94353EE021E12911F058
:104CCE00F69A01C0F698A0E0F699A1E0EA2FE795D2
:104CDE00E0E0E7955E2F40E0E0E0EDAFE09301030A
:104CEE00FE01E15BFF4F3396BF01AA89B0E0A7FD3D
:104CFE00BFEF0E949F370E9460380E943D38BF016F
:104D0E00AA89B0E0A7FDBFEF0E948E39A9A1BAA172
:104D1E00A031E7E2BE0740F00E94E338BF01A9A12F
:104D2E00BAA10E94433AEC93A9A1BAA1A83EE3E02E
:104D3E00BE0740F00E940839BF01A9A1BAA10E9486
:104D4E00A938EC93A9A1BAA1A436E0E0BE0740F0C1
:104D5E000E941539BF01A9A1BAA10E94B438EC93E3
:104D6E00A9A1BAA11A9738F00E94BF380E94483AFA
:104D7E000E94C438EC930E942039BF01A9A1BAA1A8
:104D8E000E94DA39EA89E03079F4ECE10E944C3A7B
:104D9E00E0E50E94C337EDE60E94B239E4E50E94D9
:104DAE00B739E0E50E94D039AA89A13031F4EBE59C
:104DBE000E944C3AEDE60E94C337AA89A23029F42C
:104DCE000E944F3AE8E30E94C337AA89A33049F400
:104DDE00EEE50E94B937E0E30E94BE37E7E70E9496
:104DEE00C337AA89A83011F40E94533AAA89AC306D
:104DFE0031F4EEE30E94593AECE70E94C337AA89D8
:104E0E00E1E10E942F3AE2E10E94343AE3E10E948E
:104E1E00343AE5E10E94343AEDE10E94343AEEE292
:104E2E000E94173EE02939F00E94BF380E94483A8E
:104E3E000E94C438EC93E7EAE0937A000E948A332A
:104E4E00E7E2E0937A00AA890E949D39AA89EEE0F2
:104E5E000E94343AE1E10E94173EE02911F0E1E0B0
:104E6E007E2EAA89E6E00E942F3AEFE00E94343AA5
:104E7E00E2E10E94173EE02911F0E2E07E2EAA89BF
:104E8E00E7E00E942F3AE0E10E94343A0E945C3A39
:104E9E0011F0E3E07E2E0E949433D39708F45DC0A8
:104EAE000E9403340E940834E72D0E940F3420F034
:104EBE00E8ECF0E00E94C233A0914203A13011F45D
:104ECE000E941F34E72D0E942A340E94613AAC9151
:104EDE00A13008F441C00E94683A0E944A340E94F0
:104EEE00CE3F4CF40E94613A0E94713A0E94CE3D30
:104EFE000E947B3A23C00E94843A0E946B34EF9347
:104F0E000E94843A0E947434AF91EA2379F00E9491
:104F1E00613A0E94713A0E94D33DA093A703B093C9
:104F2E00A8038093A9039093AA0308C00E94843A11
:104F3E000E947D341CF00E94863A0EC0A091A703F9
:104F4E00B091A8038091A9039091AA030E94963470
:104F5E000E94063F0E94C23304C00E94C7330E94C3
:104F6E00863AAA89AD3019F50E948138FF93EF93E6
:104F7E000E9412370E943839AF91BF910E948B3830
:104F8E003696FF93EF930E94953A0E943238AF9176
:104F9E00BF910E948B383796FF93EF930E94953AFC
:104FAE000E94203FAF91BF91EC93E0E2EDAFAA8952
:104FBE00A53141F4EEE30E94B937ECE00E94BE3712
:104FCE00E0E6EDAFAA890E949D39AA89EEE00E9423
:104FDE00343AE1E10E94173EE029B1F00E949B3A7B
:104FEE00E4E00E949F3A28F00E9481380E94A53A80
:104FFE00EC930E9494331A9728F00E94A83A0E94CC
:10500E00C438EC930E94AF3AAA89E6E00E942F3A88
:10501E00EFE00E94343AE2E10E94173EE029B1F03F
:10502E000E949B3AE2E00E949F3A28F00E9481384B
:10503E000E94A53AEC930E9494331A9728F00E948E
:10504E00A83A0E94C438EC930E94AF3AAA89E7E0CE
:10505E000E942F3AE0E10E94343A0E945C3AB1F08D
:10506E000E949B3AE1E00E949F3A28F00E9481380C
:10507E000E94A53AEC930E9494331A9728F00E944E
:10508E00A83A0E94C438EC930E94AF3AAA890E94B3
:10509E009D390E94B63A1E2EAA89E6E00E94173E5E
:1050AE000E2E0E94B63A1E2AAA89E7E00E94173EEB
:1050BE000E2E0E94B63AE12951F1E72DF0E0DE0105
:1050CE00D896AE0FBF1FEC91F0E0AF89B88D0E945D
:1050DE00913EDF01E4E6F0E00E94C93E0E94C23339
:1050EE000E9494331A9750F00E948138BF010E949B
:1050FE0094330E94ED360E94C438EC930E94B93A64
:10510E000E9494330E94DA39E7E70E94C337AA89D6
:10511E00A431B1F40E9481380E94BF3A0E94B43883
:10512E000E948B3836960E94BF3A0E94ED360E943E
:10513E00C4380E948B3837960E94BF3A0E94DA39E3
:10514E00AA89A63129F40E94533AEBE00E94AD39A8
:10515E00AA89A73129F40E94533AE0E40E94AD399E
:10516E00AA89A83129F40E94533AECE00E94AD3985
:10517E00AA89A931C9F4AB81AA2322F40E94473827
:10518E000E944F380E948138BF010E9454380E94FD
:10519E009F370E9460380E94B93A0E9454380E948C
:1051AE008E39E7E70E94C337AA89AA31F1F40E942B
:1051BE00C53AA436E0E0BE0740F00E948138BF0138
:1051CE000E94C53A0E94B438EC930E94B93A0E94EC
:1051DE00C53A0E94ED360E94C4380E948B3837962D
:1051EE00BF010E94C53A0E94DA39AA89AB3169F42F
:1051FE00ECE70E94593AE8E70E94C3370E94BF3895
:10520E000E94483A0E94C438EC93AA89AC3149F402
:10521E00E0E30E94B937EDE60E94BE37E4E50E9456
:10522E00C337AA89AF3149F4EEE30E94B937EDE6F0
:10523E000E94BE37E3E70E94C337AA89A53229F43C
:10524E000E94CA3AE5E00E94C337AA89A63229F421
:10525E000E94CA3AE8E00E94C337AA89A73229F40D
:10526E000E94CE3AE3E60E94C337AA89A83229F4F7
:10527E000E94CE3AE8E70E94C337AA89A93249F4C0
:10528E00E7E70E94B937E0E40E94BE37E8E70E94E4
:10529E00C337AA89AB3231F4E9E30E94D23AEEE089
:1052AE000E94C337AA89AC3231F4ECE70E94D23A9D
:1052BE00EDE60E94C337AA89AD3231F4E0E00E94D8
:1052CE00D53AE0E00E94C337AA89EDE10E942F3A59
:1052DE00EEE10E94173EE02921F1E3E70E94AD398D
:1052EE00E8E30E94B239AA89AD3111F4EEE501C0AE
:1052FE00E8E7DE01A65ABF4FEC930E94D83A1A9700
:10530E0048F00E94B93A0E94D83A0E94ED360E94A7
:10531E00C438EC930E94DD3ABF010E94D83A0E9435
:10532E00DA39AA890E949D39AA89E6E00E94343AA8
:10533E00E7E00E94173EE02919F0E3E70E94AD393D
:10534E00AA89EEE00E942F3AEFE00E94343AE0E1A3
:10535E000E94173EE02949F0EDE60E94AD39E9E7DB
:10536E000E94B239E4E50E94B739AA89E1E10E94B0
:10537E002F3AE2E10E94343A0E945C3A19F0E8E7D3
:10538E000E94B239AA89EFE10E942B3E0E2EE5E271
:10539E000E94263EE02161F0EDE60E94B937E8E575
:1053AE000E94BE370E94DD3ADF01EA89EF51EC938D
:1053BE00AA89AE3231F4E9E30E94B937E8E30E94DC
:1053CE00BE37AA89AF3249F4E8E70E94B937E5E063
:1053DE000E94BE37E7E70E94C337AA89A03331F493
:1053EE00E0E30E944C3AE0E50E94C337AA89A1335C
:1053FE00B1F4E3E70E94D23AE8E70E94C337A091E6
:10540E000203A43160F0E4E50E94AD39EDE60E949E
:10541E00B239E0E30E94B739EDE30E94D039AA8990
:10542E00A23341F4EEE30E94B937EBE00E94BE379F
:10543E00E0E6EDAF0E94393A0E943F3EE02111F0C6
:10544E000E94E23AAA89A33329F40E94E83AE8E3DB
:10545E000E94C337AA89A43389F4E8E70E94B937BA
:10546E00E8E30E94BE370E94DD3AA0912B03A08391
:10547E00A9A1BAA1549711F40E94E23AAA89A533C0
:10548E0049F4E8E30E94B937E0E30E94BE37E4E551
:10549E000E94C337AA89AC3549F4E7E70E94B937B1
:1054AE00E9E30E94BE37E9E30E94C337AA89AD350E
:1054BE0009F086C0ACADA83008F044C0E7E70E9402
:1054CE00D53A0E94DD3AACADA083E7EAE0937A00CC
:1054DE000E945D33E0935103F0935203E7E2E093B1
:1054EE007A000E94EC3AA83EE3E0BE0740F00E942C
:1054FE000839BF010E94EC3A0E94A938EC930E9431
:10550E00EC3AA436E0E0BE0740F00E941539BF0128
:10551E000E94EC3A0E94B438EC930E94EC3A1A972F
:10552E0050F00E94BF38BF010E94EC3A0E94ED3647
:10553E000E94C438EC930E942039BF010E94EC3ABD
:10554E000E94DA39ACADA830E1F4E6E70E94593A90
:10555E00E8E30E94F13ADF01E0914703E1700E9417
:10556E008B383E96DF01E0914703E695E1700E948D
:10557E008B383F96DF01E0914703E695E695E170A3
:10558E00EC93ACADA930E1F40E94E83AE0E30E945E
:10559E00C3370E94AC361A974CF00E941539BF01E2
:1055AE000E94AC360E949F370E9460380E94BF381E
:1055BE00BF010E94AC360E948E39E7E70E94E239A5
:1055CE00AA89AE3509F0BBC1E0914903E030D1F4B0
:1055DE000E944F3AEBE00E94C3370E946D37EA30CB
:1055EE0048F00E94BF38BF010E946D370E94F33A07
:1055FE000E9460380E942039BF010E946D37F0E092
:10560E000E946038A0914903A130F1F4E0E30E94BA
:10561E00F63AEBE00E94C3370E947237EA3048F048
:10562E000E941539BF010E9472370E94F33A0E9400
:10563E0060380E94BF38BF010E947237F0E00E94AE
:10564E006038E7E70E94E239A0914903A230F1F4F5
:10565E00E0E30E94B937E3E70E94F93A0E947737F8
:10566E00EA3048F00E941539BF010E9477370E9438
:10567E00F33A0E9460380E94BF38BF010E9477370C
:10568E00F0E00E946038E7E70E94E239A0914903FA
:10569E00A330E9F4EEE30E94F63AECE00E94F13A10
:1056AE00BF010E947C37DF010E948B390E94BF38F8
:1056BE00BF010E947C37DF010E949F370E94603835
:1056CE000E942039BF010E947C370E946038A09151
:1056DE004903A430E9F4EEE30E94F63AEBE00E94AF
:1056EE00F13ABF010E948637DF010E948B390E947A
:1056FE00BF38BF010E948637DF010E949F370E948C
:10570E0060380E942039BF010E9486370E9460389F
:10571E00A0914903A530D1F5E3E70E94B937EBE03C
:10572E000E94BE370E94A437E83EA3E0FA0744F079
:10573E000E94E338BF010E94A437DF010E9488391E
:10574E000E94A437E436A0E0FA0744F00E9408391C
:10575E00BF010E94A437DF010E948B390E94A4373B
:10576E003A9754F00E941539BF010E94A437DF0109
:10577E000E949F370E9460380E94BF38BF010E946E
:10578E00A4370E946038EEE30E94E239A0914903EB
:10579E00A63059F5E8E70E94B937E0E00E94F93AE1
:1057AE000E948B37E436A0E0FA0744F00E94E338FB
:1057BE00BF010E948B37DF010E948B390E948B370D
:1057CE003A9754F00E940839BF010E948B37DF01CF
:1057DE000E949F370E9460380E941539BF010E94B7
:1057EE008B370E9460380E94FC3AA0914903A73083
:1057FE0059F5E8E70E94B937E1E00E94F93A0E94B4
:10580E009037E436A0E0FA0744F00E94E338BF0177
:10581E000E949037DF010E948B390E9490373A9791
:10582E0054F00E940839BF010E949037DF010E9498
:10583E009F370E9460380E941539BF010E94903731
:10584E000E9460380E94FC3AA0914903A83059F595
:10585E00E8E70E94B937E2E00E94F93A0E949537D4
:10586E00E436A0E0FA0744F00E94E338BF010E943C
:10587E009537DF010E948B390E9495373A9754F085
:10588E000E940839BF010E949537DF010E949F37A1
:10589E000E9460380E941539BF010E9495370E9400
:1058AE0060380E94FC3AA0914903A93009F047C024
:1058BE00ECE70E94D23A0E94C231A031E7E2BE0765
:1058CE0038F00E94D6380E94C2310E94433AEC93BF
:1058DE000E94C231A83EE3E0BE0740F00E94E838C5
:1058EE00BF010E94C2310E94A938EC930E94C231BE
:1058FE00A436E0E0BE0740F00E94E338BF010E94EC
:10590E00C2310E94B438EC930E94C2311A9750F003
:10591E000E940839BF010E94C2310E94ED360E94DA
:10592E00C438EC930E941539BF010E94C2310E9407
:10593E00DA39E4E50E945139E7E70E94E239AA8993
:10594E00AF3569F50E94C036AFE8B3E00E9416325B
:10595E00AB81AA2342F4E0918F03F09190030E9451
:10596E00D83D0E944F380E948138BF010E945438A2
:10597E000E948B390E94B93A0E9454380E949F3778
:10598E000E9460380E94DD3ABF010E9454380E9486
:10599E008E39EEE50E94AD39E1E00E94B239AA8956
:1059AE00A03631F4E8E30E94D53AEDE00E94C33709
:1059BE00AA89A13631F4E8E70E94593AEEE30E9433
:1059CE00C337AA89A23661F4E8E30E94B937FE0113
:1059DE00E15BFF4F3696A0913203A083E0E1EDAF7D
:1059EE00AA89A33699F4E8E30E94D53A0E94EE35CF
:1059FE00EA17FB0718F4ECE00E94C3370E94EE355D
:105A0E000E94F53519F0EBE00E94C33731E03031DA
:105A1E0008F089C00E94273AEC91E03021F40E94F0
:105A2E00273AEFE3EC930E94273AAC91A63021F48B
:105A3E000E94273AEDE7EC930E94273AAC91A130F1
:105A4E0021F40E94273AE6E0EC930E94273AAC91AB
:105A5E00A23021F40E94273AEBE5EC930E94273AFC
:105A6E00AC91A33021F40E94273AEFE4EC930E940C
:105A7E00273AAC91A43021F40E94273AE6E6EC9343
:105A8E000E94273AAC91A53021F40E94273AEDE608
:105A9E00EC930E94273AAC91A73021F40E94273A4A
:105AAE00E7E0EC930E94273AAC91A83021F40E94D3
:105ABE00273AEFE7EC930E94273AAC91A93021F4F4
:105ACE000E94273AEFE6EC930E94273AAC91AA3057
:105ADE0021F40E94273AE0E0EC930E94273AAC9121
:105AEE00AB3021F40E94273AE1E0EC930E94273A72
:105AFE00AC91AC3021F40E94273AE8E0EC930E947E
:105B0E00273AAC91AD3021F40E94273AE0E4EC93B1
:105B1E000E94273AAC91AE3021F40E94273AE9E078
:105B2E00EC933F5F74CFE0910103E695E695E1704B
:105B3E000E941C370E94003B0E94053B0E94003BC6
:105B4E000E940D3B0E94003B0E94183B0E94003BAE
:105B5E000E94EB390E941F3B0E94223B0E941F3B7A
:105B6E000E94273B0E941F3B0E942C3BEA2BEFAF6B
:105B7E00FE01FE9632960F01E09101030E942C3B2E
:105B8E000E941C370E94313B0E94053B0E94313B14
:105B9E000E940D3B0E94313B0E94183B0E94363BF7
:105BAE000E94EB390E943B3B0E94223B0E943B3BF2
:105BBE000E94273B0E943B3B0E942C3B0E943E3B97
:105BCE0033960F01E0910103E695E1700E941C37B8
:105BDE000E94363B0E94053B0E94363B0E940D3BC5
:105BEE000E94363B0E94183B0E94313B0E94EB39CB
:105BFE000E94443B0E94223B0E94443B0E94273B52
:105C0E000E94443B0E942C3B0E943E3B34960F0167
:105C1E00FE01E95AFF4FE081E1700E941C370E949D
:105C2E00473B0E94053B0E94473B0E940D3B0E9452
:105C3E00473B0E94183BE52F0E94EB39EA2BAE2F13
:105C4E00E52F0E94223BEA2BAE2FE52F0E94273B29
:105C5E00EA2BAE2FE0910103E1700E943E3B359698
:105C6E000F010E944C3BE1700E941C370E944C3B7E
:105C7E000E94513B0E944C3B0E94573B0E944C3B62
:105C8E000E942C3B0E94603B0E94663B0E946A3B36
:105C9E000E946D3B0E946A3B0E94743B0E946A3BCD
:105CAE000E947B3B36960F010E947E3BE1700E9464
:105CBE001C370E947E3B0E94513B0E947E3B0E94FD
:105CCE00573B0E947E3B0E942C3B0E94603BE2951C
:105CDE000E94EB390E94833B0E946D3B0E94833BE6
:105CEE000E94743B0E94833B0E947B3B37960F01C0
:105CFE00E52F0E948A3B0E941C370E947E3B0E9429
:105D0E00053B0E947E3B0E940D3B0E947E3B0E9403
:105D1E00183B0E948F3B0E94EB390E94943B0E94DD
:105D2E00223B0E94943B0E94273B0E94943B0E9480
:105D3E002C3B0E943E3B38960F010E94973BE17030
:105D4E000E941C370E94973B0E94513B0E94973B3A
:105D5E000E94573B0E94973B0E942C3B0E94603B47
:105D6E000E949C3B0E94EB390E94943B0E946D3B2B
:105D7E000E94943B0E94743B0E94943B0E947B3B8A
:105D8E0039960F010E94A13BE1700E941C370E94C0
:105D9E00A13B0E94513B0E94A13B0E94573B0E9497
:105DAE00A13B0E942C3B0E94603BEE1FE0E0EE1FE9
:105DBE000E94EB390E94A63B0E946D3B0E94A63BBF
:105DCE000E94743B0E94A63B0E947B3B3A960F01B9
:105DDE00E42FE295E1700E941C370E94A13B0E94C5
:105DEE00053B0E94A13B0E940D3B0E94A13B0E94DD
:105DFE00183B0E94473B0E94EB390E94AD3B0E942C
:105E0E00223B0E94AD3B0E94273B0E94AD3B0E946D
:105E1E002C3B0E943E3B3B96BF010E94B03BE17083
:105E2E000E941C370E94B03B0E94513B0E94B03B27
:105E3E000E94573B0E94B03B0E942C3BE295E07FB4
:105E4E00EA2B0E2EA0E035FCA1E0EA2FEE0FEE0FAE
:105E5E00EE0FE0290E94B53BE2950E94BB3B0E94EB
:105E6E00B53B0E94743BEA2B0E94B53B0E948A3BD5
:105E7E00EA2BDB01EC93FE01FE963C960F01FE0130
:105E8E00E05BFF4FE0810E942C3B0E941C37FE011D
:105E9E00E05BFF4FE081E695E6950E94C03B0E94D5
:105EAE00B53B0E94C43B0E94B53BE1700E94CB3BC8
:105EBE00E42F0E94663BEA2BAE2FE42F0E94D03BCC
:105ECE00AE2FE42F0E94D33BE42FE695E1700E94A3
:105EDE003E3B3D960F01E42F0E948A3B0E941C37E9
:105EEE000E94D83BE2950E94C03BAE2F0E94D83B49
:105EFE000E940D3B0E94D83B0E948A3B0E94CB3BE6
:105F0E000E94D83B0E94663BEA2BAE2F0E94D83BE4
:105F1E000E94D03BAE2F0E94D83BE6950E94D33B09
:105F2E000E94D83BE1700E943E3B3E960F01E42F4B
:105F3E000E949C3BE1700E941C37EDAD0E94C03B5D
:105F4E00AE2FEDAD0E94C43BAE2FEDADE695E695BE
:105F5E00E1700E94CB3BE0910103E2950E94EB3988
:105F6E00EA2BAE2FE42FEE1FE0E0EE1F0E94BB3BAC
:105F7E00AE2FEDAD0E942C3BEE0FEA2BAE2FEDAD0A
:105F8E000E947B3B3F960F01EDAD0E948A3B0E9423
:105F9E001C370E94DD3BE2950E94C03BAE2F0E9453
:105FAE00DD3B0E940D3B0E94DD3B0E948A3B0E941E
:105FBE00CB3B0E94E23B0E94663BEA2BAE2F0E9437
:105FCE00E23B0E94D03BAE2F0E94E23BE6950E9440
:105FDE00D33B0E94E23BE1700E943E3B70960F0164
:105FEE00EDAD0E949C3BE1700E941C370E94E23B8B
:105FFE00E2950E94C03BAE2F0E94E23B0E940D3BF9
:10600E000E94E23B0E948A3B0E94CB3B0E94DD3BFA
:10601E000E94663BEA2BAE2F0E94DD3B0E94D03BD6
:10602E00AE2F0E94DD3BE6950E94D33B0E94DD3BE6
:10603E00E170EA2BD001EC9333FE0DC031E031312B
:10604E0050F4E32FF0E0DE01DE96AE0FBF1FEFEF50
:10605E00EC933F5FF4CF0E94E73B3D3078F40E9413
:10606E00ED3BA2E5B8E00E94F53DE17011F45D98BC
:10607E0001C05D9A0E94F43B3F5FEFCF0E94FC3B54
:10608E003D3078F40E94ED3BA0E3B8E00E94F53D70
:10609E00E17011F45D9801C05D9A0E94F43B3F5F80
:1060AE00EFCF0E94FC3B3D3078F40E94ED3BA2E026
:1060BE00B8E00E94F53DE17011F45D9801C05D9A63
:1060CE000E94F43B3F5FEFCF0E94FC3B3D3078F4E3
:1060DE000E94ED3BA6E0B8E00E94F53DE17011F4A0
:1060EE005D9801C05D9A0E94F43B3F5FEFCF0E9426
:1060FE00FC3B3D3058F50E94053CA0913F030E94A9
:10610E00F633A0913E030E943035A0E0F099A1E055
:10611E000E94BA3461F0ECE0E31BA2E1B8E00E9409
:10612E00F53DE17011F45D9801C05D9A0BC0ECE095
:10613E00E31BA0E1B8E00E94F53DE17011F45D981B
:10614E0001C05D9A0E94F43B3F5FD3CFA0913F0305
:10615E000E94F633A0913E030E943035A0E0F099E4
:10616E00A1E00E94BA3419F0E1E0E0933E03E09121
:10617E003F03E03019F4E0E0E0933E035D9A84E0E3
:10618E008A95F1F7289A84E08A95F1F7289884E0A9
:10619E008A95F1F731E03A3088F40E94053CE9E047
:1061AE00E31BA0E4B1E00E94F53DE17011F45D98AF
:1061BE0001C05D9A0E94F43B3F5FEDCF21E021319B
:1061CE00D8F431E03930B0F40E94053CE22FF0E013
:1061DE00DE01DE96AE0FBF1FAC91E8E0E31B0E941E
:1061EE00E43DE17011F45D9801C05D9A0E94F43BAC
:1061FE003F5FE8CF2F5FE3CF5D9A85E28A95F1F797
:10620E00289A84E191E00197F1F70E94E733A92DD6
:10621E000E940A3CAB2D0E940A3CAA2D0E940A3C09
:10622E000E9404370E2A0E944D35E0E0F0E060E057
:10623E007FEB0E94C23D0E2A0E9496350E2A0E94C6
:10624E00B034E02929F0E0E0E0936B03E0936C03B7
:10625E00F09B03C0E0E0E0933F03A82DE4E60E942C
:10626E003A3E0E2EA0E0F099A1E00E94AD3329F047
:10627E000E945933F09AE89433F80C949F06FFCF9E
:10628E00AA93E091C000E072E1F3E881E093C600CA
:10629E0021960895A0915503B09156030895A091AB
:1062AE00BF03B091C0038091C1039091C2030895C2
:1062BE00E0E0F0E061EE75E40E945D3D0895E0914E
:1062CE006103F09162030895662777270E94853C4B
:1062DE000E94593F0895E0916D03F0916E03089569
:1062EE00A091C703B091C8038091C9039091CA03CE
:1062FE000895E0E0F0E060E271E40895A09161039A
:10630E00B09162030895E0E0F0E00E94633E0895CC
:10631E00A0916D03B0916E030895E091EB03F0919F
:10632E00EC036091ED037091EE0308950E944C3CD6
:10633E00ED93FC930895A091DB03B091DC03809163
:10634E00DD039091DE030895E0E0F0E06AE774E487
:10635E000E940F3DDF01CB01ABCFA091D703B091CF
:10636E00D8038091D9039091DA030895E0E0F0E02C
:10637E0060E070E00895A0917503B09176030895E2
:10638E000E94773F0E94B83C0895A091FB03B09104
:10639E00FC038091FD039091FE030895E0917B0331
:1063AE00F0917C0360917D0370917E030895A4E6C5
:1063BE00B0E080E090E00E94993EDF01CB01E091D9
:1063CE00D703F091D8036091D9037091DA030E943C
:1063DE00723F0895E0917303F09174030895E09372
:1063EE007303F09374030895A091F303B091F40333
:1063FE008091F5039091F6030895E093F303F093E3
:10640E00F4036093F5037093F6030895A0917B0354
:10641E00B0917C0380917D0390917E0308950E943C
:10642E004E3CED93FC930895E0E0F0E061EE75E4F0
:10643E000E940F3D0895A091DF03B091E00380917B
:10644E00E1039091E2030895E7EEF3E0E093910308
:10645E00F09392030895E091DF03F091E0036091D1
:10646E00E1037091E2030895E091E303F091E403F8
:10647E006091E5037091E6030895A091C303B09176
:10648E00C4038091C5039091C6030895E093C3039E
:10649E00F093C4036093C5037093C6030895A0914F
:1064AE00CB03B091CC038091CD039091CE03089590
:1064BE00E091C303F091C4036091C5037091C603CC
:1064CE000895A091D303B091D4038091D5039091F8
:1064DE00D6030895E0917703F091780360917903E4
:1064EE0070917A030895E0937703F09378036093A5
:1064FE00790370937A030895EDDFAFE5B0E00E9463
:10650E00983F0895A0917703B09178038091790315
:10651E0090917A030895EDDE0E940F3D0895E0E01C
:10652E000E943A3E0E2E0895A091AB03B091AC039B
:10653E008091AD039091AE0308950E22A091260393
:10654E00ECE30E94353E0895A0916B03B0916C036D
:10655E000895A0916903B0916A03D5CEE0916903C5
:10656E00F0916A030895A4E6B0E00C940F3CE7EABC
:10657E00E0937A00A4E00C94E603EF2FF0E06E2E89
:10658E00E7E2E0937A000895E7EAE0937A00A3E069
:10659E000E94E603EF2FF0E09E2EE7E2E0937A00F2
:1065AE000895E7EAE0937A00A1E00E94E603EF2F58
:1065BE00F0E0BE2EE7E2E0937A000895E0E0F0E02E
:1065CE000E94A03F0895EBE0E0930404E8EBE09313
:1065DE0005040895E0938103F09382030895E093F8
:1065EE008303F09384030895E0935903F0935A03C1
:1065FE0008950E940D3E0E94853C0E94593F0895C9
:10660E0078DE0E945D3D0895E0935F03F093600392
:10661E000895E0937B03F0937C0360937D03709366
:10662E007E030895E0936903F0936A030895ADE540
:10663E00B0E00E94883F0895E0936F03F0937003DB
:10664E000895E0933903E0E0E09318040895E09193
:10665E000304F0E0E0939903F0939A03E0910404AD
:10666E00F0E0EADFE0910504ECCFE0E0E093FF0319
:10667E00E0930004E0930104E0930204E09303042A
:10668E00A2CFE0E0E0930604E0930704E093080451
:10669E00E0930904E09318040895E0939903F093AE
:1066AE009A030895AAE0B0E00C940F3C0E94E60312
:1066BE000E94023E0E94FE3D0895E7EAE0937A00B2
:1066CE00A0E00E94E603EF2FF0E00895E887F98737
:1066DE006A877B870895E0915903F0915A030895D4
:1066EE00E885F9856A857B850895E7E2E0937A006F
:1066FE008AE48A95F1F708958AE48A95F1F7E7EA34
:10670E00E0937A000895A7E00E94E603EF2FF0E0F1
:10671E00E0934F03F09350030895A0914F03B0916F
:10672E0050030895E2E3F0E00E94633E0E2E0895BA
:10673E00ADA1BEA1F7CFEEE1F0E00E945D3E0E2EC0
:10674E00A52DE1E00E943A3E0E220895E0E00E945F
:10675E00173EE0210895EAEFF0E00E94633E0E2E10
:10676E00A52DE1E00E943A3E0E220895E4E00E943B
:10677E00353EE0210895E0934F03F09350030895C2
:10678E00E0E0E0934F03E09350030895E4E00E94AD
:10679E00173E0E2E0895AEA5E5E00E94173E089511
:1067AE00AA2DEAE00E94353E0E2E0895A0E0F3FCDD
:1067BE00A1E0E0E00E94173E0E22A02FE3E608952E
:1067CE00A62DEAE00E94353E0E2E0895ADDEE2E0E3
:1067DE00F0E060E070E00E94813EE0210895E1E08B
:1067EE000E94173E0E2E0895A0911403AFCFE3E042
:1067FE000E94173E0E2E0895E0914F03F091500324
:10680E000895F297ADE7B0E00E94913E0F01089512
:10681E00F0E0DE01D496AE0FBF1FEC91F0E0D00198
:10682E000E94C93EA8DF79DFA93CE0E0BE070895CB
:10683E00EF89F88D72DF0E94913EDF01E4E1F0E016
:10684E000E94C93E98CFF0E0DE01D896AE0FBF1F72
:10685E00EC91F0E062DF0E94913EDF01E4E6F0E0B1
:10686E000E94C93E88CFE12FF0E0DE01D096AE0F38
:10687E00BF1F0895A091A303B091A4038091A50317
:10688E009091A6030895E8EEF3E060E070E00E94B8
:10689E00063FDF01CB01B0DF662777270895EC9125
:1068AE00F0E0A0E4BCE90E94C93EE4DF662777274A
:1068BE000895E093A303F093A4036093A50370934C
:1068CE00A6030895D7DFDFCF0E94D33DE5E0F0E0C9
:1068DE0060E070E00E94893E08950E94D33DE4E19D
:1068EE00F0E060E070E00E94813E08950E94D33D8A
:1068FE00A431E0E0BE07E0E08E07E0E09E070895D9
:10690E00E091AB03F091AC036091AD037091AE03D7
:10691E00A0E5B4E180E090E00E94C43ECACFE8EE6C
:10692E00F3E060E070E00895A02FE3E60E94353EAC
:10693E000895A0E0F0FCA1E009CFEFDEE0E0F0E08A
:10694E000E943F3E0895E89425F8E0E0E093280386
:10695E000895E3DED8CC0E22A0E022FCA1E0E1E017
:10696E000E94173E0895E1E00E94173EE02108952F
:10697E00A0E025FCA1E033CFACA5E3E00E941C3ED5
:10698E00E0210895E0933603DECF0E2EADA1BEA119
:10699E00E0E0F0E00E943F3E0E220895A0E021FCD0
:1069AE00A1E0E0E00E94173E0895E0910403F0E0BC
:1069BE003597B3DE0E945D3E0E2EE0913503B4DDB9
:1069CE00FF27662777270895A0E022FCA1E0BECE20
:1069DE00EF8DF8A1A885B9858A859B8566277727CF
:1069EE000E94813E0E2EEAE0F0E060E070E00E9430
:1069FE00893E089575DEAF8DB8A1882799270E942C
:106A0E00D33D0895A630E0E0BE07E0E08E07E0E05B
:106A1E009E070895A0918103B09182030895E0919D
:106A2E008103F09182030895EF8DF8A1A885B985B1
:106A3E008A859B85662777270895EF89F88D0E94B2
:106A4E00633F662777270E94853C0E94C83D0E2E25
:106A5E000895E0E00E94173E0E2208955EDEEAE001
:106A6E000E94B93E0895EF89F88D0E94633F662714
:106A7E0077270E94853C84CCA0918303B091840338
:106A8E000895E0918303F091840308950E94633F7B
:106A9E000895662777270E94853C08950E945E3FE1
:106AAE00AF89B88D882799270E94743F69CC0E94C0
:106ABE000D3E0E94853C0895EAE0F0E00E94DC3E27
:106ACE005ACEEFA131DDFF27662777270895E09391
:106ADE008B03F0938C030895EFA1F0E025DD0E9467
:106AEE000D3E0E94D33D08950E94BF3EA0918B03A0
:106AFE00B0918C030895E0918B03F0918C0308956F
:106B0E00AFA1BB27E091AB03F091AC036091AD0355
:106B1E007091AE030E94123E0E94D33D0895ADA126
:106B2E00BEA1F1CBA0E0F099A1E0E1E00E94173EFA
:106B3E0004CD0E22A02FE3E60E94173EE021089519
:106B4E000E2EA0912603ECE30E94353E0E220895F0
:106B5E000E94A03FA1E0B0E00C940F3CE091D7035F
:106B6E00F091D8036091D9037091DA03A1E4B0E0FB
:106B7E000E944E3CEDCFA9E4B0E00E944E3CE8CF1F
:106B8E0029DCABE4B0E0E4CF0E94A83FA1E0B0E086
:106B9E000C940F3CE0917503F0917603ADE5B0E0F7
:106BAE000E94A03F0895EAE00E943A3E0E2E0895FC
:106BBE00AB2DEAE00E94353E0E2EA0E027FCA1E0B0
:106BCE0048CFE0913203F0E0E15EFC4F0895E98D8D
:106BDE00FA8D0E94023EA62DB0E008950E94573E07
:106BEE000E2EA62DEAE00E943A3EE0210895A92D30
:106BFE00EAE00E94353E0E2E0895E0910D03F0E07E
:106C0E00E85FFC4F0895E0915F03F09160030895F3
:106C1E00A02FE3E60E94173EE0210895E0913B038A
:106C2E00EF5FE0933B03E0913A03A0913B03EA1739
:106C3E000895E0931803F0E03ADFACE5BFE882E296
:106C4E0090E40E940F3DA3ECB5EF88E490E40E941F
:106C5E000F3DAFE5B3E06ACBA0910E03E8E10E94D1
:106C6E00173E0E2EAF8DB8A10895E0211E2EA091D5
:106C7E000E03E4E20E94173E0E2EAF8DB8A10895CA
:106C8E00E0211E2AA0910E03E0E30E94173E0E2E75
:106C9E00AF8DB8A108950E945D3E0E2EA0E023FC9C
:106CAE00A1E00895A0915F03B09160030895ACDC5C
:106CBE00AADFEFDEDF01CB01ECE5FFE862E270E474
:106CCE000E945D3DDF01CB01E3ECF5EF68E470E47B
:106CDE000E945D3DA8E1B3E00E944C3CEC93089508
:106CEE00A0917303B09174030895E0912B03F0E02B
:106CFE00E65BFC4FA0810895A0912B03B0E0A65B4C
:106D0E00BC4FEC910895A0913203B0E0A15EBC4F50
:106D1E00EC910895AA89E3E60E94173E0E2E57CFF6
:106D2E00E1E00E94803FEA1B0E94D33F0895E0916C
:106D3E009903F0919A03BBDE0E94683F08950E946A
:106D4E00683F08950E945E3F0895A0919F03B09101
:106D5E00A0030895F7DFA0E0B0E080E09FE3089580
:106D6E00E093DB03F093DC036093DD037093DE03AB
:106D7E0008958CDED0CBE6DFAFE8B3E050CBE0E099
:106D8E000E94173E0E2E0895EA1BFB0B90DEDF01CC
:106D9E00CB01EAE9F9E969E271E40E945D3DDF01A8
:106DAE00CB01E0E0F0E068E571E4EACAEE0FFF1F08
:106DBE00A0E0B4E00E947D3FE7CFE091BB03F091ED
:106DCE00BC036091BD037091BE030895EAE0F0E04C
:106DDE000E94C93E0895A091BB03B091BC0380915F
:106DEE00BD039091BE030895E093B703F093B803EB
:106DFE006093B9037093BA03089596DBB7DA0E94D5
:106E0E00893E0895EB8DFC8DA885B9858A859B8575
:106E1E00662777270895A885B9858A859B85089565
:106E2E00E0935D03F0935E030895E795E0E0E79548
:106E3E00AE2F08950E944731A0914F030C94473115
:106E4E000E944731E0915E03AE2F0E944731A09120
:106E5E005D030C944731F0E0AE0FBF1FE0911A03B3
:106E6E00F0E00895F0E0AE0FBF1FE0914103F0E0B7
:106E7E00AE0FBF1FE091420308950E944731A091CB
:106E8E0016030E944731A09117030C9447310E94BC
:106E9E004731A0911A030C9447310E944731A091BB
:106EAE001B030C944731A1E00E944731A6E30C94DA
:106EBE0047310E944731A0915D030C9447310E94E7
:106ECE004731A0E00E944731A0E00895A6E3B0E06C
:106EDE000E948C3F0895A7E3B0E00E948C3F089576
:106EEE00A8E3B0E00E948C3F0895A1E5B0E00E94B7
:106EFE00883F0895AC85BD858E859F850895A3E551
:106F0E00B0E00E94883F0895A7E5B0E00E94883F58
:106F1E000895A9E5B0E00E94883F0895ABE5B0E082
:106F2E000E94883F0895A091A103B091A2030895F5
:106F3E00EAE0F0E00E94DC3E0895A5E5B0E00E9494
:106F4E00883F0895DE01A05BBF4FEC930895EAE001
:106F5E00DE01AE5ABF4FEC930895DE01AD5ABF4F1E
:106F6E00EC930895DE01AC5ABF4FEC930895DE0109
:106F7E00AB5ABF4FEC930895DE01AA5ABF4FEC9364
:106F8E000895EAE0DE01A95ABF4FEC93DE01A85A3C
:106F9E00BF4FEC93DE01A75ABF4FEC93DE01A65A0A
:106FAE00BF4FEC93DE01A55ABF4FEC93DE01A45AFE
:106FBE00BF4FEC93DE01A35ABF4FEC93DE01A25AF2
:106FCE00BF4FEC93089559E0E0913803E170EE0F56
:106FDE00AE2FE0913803E695E170EE0FEE0FEE0F57
:106FEE00EA0F0E2E0895E0913803E695E695E170CE
:106FFE00AE2FE0E0F5FCE1E0EA2BEE0FEE0FE00D38
:10700E004E2F08955E2FE0913803E170EE0FAE2FF4
:10701E00E0913803E695E170EE0FEE0FEE0FEA0FFA
:10702E000E2EE1CFE295E07FEE0FEE0F0895E0E039
:10703E0020FCE1E0E09301035DCFAA30E0E0BE0763
:10704E00E0E08E07E0E09E0708956EDAEAE0F0E0F9
:10705E0060E070E008950E94063FDF01CB01EAE098
:10706E00F0E060E070E00E94203F0895FE01E15BD9
:10707E00FF4F34960895DE01AE5ABF4FEC9308953C
:10708E00E0918D03F0918E030E94D83DDF0150CF29
:10709E00E0938F03F09390030895A0918F03B09126
:1070AE0090030895FE01E15BFF4F3196BF01F5DFBE
:1070BE003FCFDF01EAE0F0E00E940E3FDB01EC93F0
:1070CE000895FE01E15BFF4F3296BF01E6DFEAE075
:1070DE00F0E00E940E3FDB01EC930895E0912B034C
:1070EE00A3E9B3E0F0E0EE0FFF1FAE0FBF1F0E944B
:1070FE00553F0895FE01E15BFF4F35960895E4E696
:10710E00F0E060E070E00895EC93FE01E15BFF4F6C
:10711E000895F0DEEAE0F0E060E070E00895A0E0AF
:10712E0020FCA1E0EA2FE295E07F4E0F0895A0919A
:10713E005703B09158030895FE01E15BFF4F3D9652
:10714E00BF01F5CFE8EEF3E00E94C93EDF01EAE0B1
:10715E00F0E00E940B3FDB010895E4E6F0E00E94B0
:10716E00C93EDF01EAE0F0E00E940B3FDB0108952B
:10717E00FE01E15BFF4F3E960895DF01EAE0F0E08D
:10718E000E940B3FDB0108950E940B3FDB01EC9345
:10719E000895E2E0DE01A95ABF4FEC930895FE0177
:1071AE00E15BFF4F3996BF010895BB27EAE0F0E09F
:1071BE000E940E3FDB010895FE01E15BFF4F3B96FF
:1071CE000895FE01E15BFF4F3A9608950E94E13E5D
:1071DE00DF01CB01EAE0F0E060E070E00E941C3FCE
:1071EE000895A031E7E2BE07E0E08E07E0E09E07DB
:1071FE000895A83EE3E0BE07E0E08E07E0E09E07BC
:10720E000895FE01E15BFF4F3C960895A436E0E041
:10721E00BE07E0E08E07E0E09E070895FE01E15B09
:10722E00FF4F3D9608956ED9EAE0F0E060E070E021
:10723E000895FE01E15BFF4F3F960895DE01A85AC7
:10724E00BF4FEC93E4E7DE01A75ABF4FEC930895CE
:10725E00A091AF03B091B0038091B1039091B203AE
:10726E0008954DDFF8CEF4DFEAE0F0E060E070E084
:10727E000895E091AF03F091B0036091B103709166
:10728E00B2030E94DC3DDF01CB01EAE0F0E060E0FA
:10729E0070E00895DE01A35ABF4FEC930895E0E429
:1072AE00DE01A45ABF4FEC930895E091AF03F09125
:1072BE00B0036091B1037091B2030E94DC3DDF0117
:1072CE00CB010895E0E4DE01A55ABF4FEC9308957B
:1072DE00E0E4DE01A65ABF4FEC930895E4E4DE012C
:1072EE00A65ABF4FEC93E1E0DE01A55ABF4FEC93D7
:1072FE000895A0918903B0918A0308950E94DC3EFF
:10730E00D8CEE8EEF3E0FACFE4E6F0E0F7CFEAE02D
:10731E00F0E00E940E3FDB01EC930895BF01E09177
:10732E008903F0918A030E94D83D0895E5E00E94FA
:10733E00173E0E2E0895E0E5DE01A65ABF4FEC93E0
:10734E000895A0919103B09192030895DE01A85A79
:10735E00BF4FEC930895DE01A75ABF4FEC930895EB
:10736E00DE01A65ABF4FEC930895EDA1FEA1F6954E
:10737E00E7950895E8ECF0E00E94C93EFECEE4E108
:10738E00F0E00E94C93EF9CEED8DFE8DF695E795A3
:10739E000895DE01A55ABF4FEC930895A0916303A3
:1073AE00B09164030895EAE0F0E0EECEDE01A45A57
:1073BE00BF4FEC930895DE01A25ABF4FEC93089590
:1073CE000E944B3E0E2EAFCDE170EE0FEE0FEE0F84
:1073DE000895ECE7C0DFAFCFAEA5E4E00E94173E04
:1073EE00AE2FE0E020FCE1E0EA230895AE2FE0E0CE
:1073FE0020FCE1E0EA230895ECE7D8DFE0E54ACF90
:10740E00E7E7D4DFE9E346CFF0E00E94513EEECF4E
:10741E00E4E10E943A3EE0210895E0932B03E8E771
:10742E0095CF99DFEAE09CDFE9E7B3DFE0E5BEDF69
:10743E00E0E530DFEAE0BFDFE1E0E0933F030895EF
:10744E00E32FF0E0DE01A15BBF4FAE0FBF1F08952B
:10745E000E94173E0E2EAA8908950E94173E0E2AEC
:10746E00AA890895AA89E2E30E94173E0E2EA9A1C9
:10747E00BAA1E4EAF1E00895E0E1F7E20E94C93E24
:10748E007CCEBF01A9A1BAA1A1CC6CDDE9E76FCD7D
:10749E00EDE668DDE3E76BCDE9E364DDE0E567DDAE
:1074AE00EEE36ACD5FDDE7E762CDE3E10E94173ED2
:1074BE00E0290895E72DF0E0DE01D096AE0FBF1F54
:1074CE000895A091A703B091A8038091A90390916C
:1074DE00AA030895EC91F0E0A0E4BCE90E94C93E35
:1074EE00F0DF662777270895E093A703F093A803AC
:1074FE006093A9037093AA030895E3DFC4C9E091D2
:10750E00AB03F091AC036091AD037091AE03A0E5B7
:10751E00B4E180E090E00E94C43EE6CF7CDCEAE07D
:10752E00F0E060E070E0089567D9F695E79523C91D
:10753E00EDAFF3D8A436E0E0BE070895BF01EDD855
:10754E000CCEFE01E15BFF4F3696BF01E6D83ECC76
:10755E00FE01E15BFF4F3796BF01DFD824CFA0912C
:10756E00420301CAFE01E15BFF4F3696BF0108954B
:10757E00BF01A0917103B09172030895A0915B03B6
:10758E00B0915C030895E8E5EDDCE4E5F0CCEDE6C2
:10759E00E9DCE8E3ECCCE6DCE0E5E9CCE3DCEEE5C7
:1075AE00E6CCA0916703B09168030895FE01E15BFC
:1075BE00FF4F37960895E0E0F9DEE1E76BDEE1E795
:1075CE00FACEE3E7CFDCE4E7D2CCA0915103B09141
:1075DE0052030895D1DC22CEF0E0DF01A9CCC2DC4B
:1075EE00ECE7C5CCC4DCEBE0C7CCE3E653DEE9E365
:1075FE00E2CEFE01EC5AFF4FE0810895E295EF7066
:10760E00E695E1700FDDEA2BAE2F0895E295EF704F
:10761E00E695E695E170E295E07FEE0FEA2BAE2F50
:10762E000895E295E170E295E07FEA2BAE2F089582
:10763E00EA2BAE2FDECFE695E170EE0FEE0F08953A
:10764E00E695E695E170EE0F0895E695E695E695DA
:10765E00E1700895FE01EB5AFF4FE0810895FE019F
:10766E00EA5AFF4FE0810895EA2BAE2FF8CFEA2BAE
:10767E00D001EC93FE01FE960895EA2BAE2FEACFD1
:10768E00FE01E85AFF4FE0810895FE01E45AFF4FD4
:10769E00E0810895E695E170C5DCEA2BAE2F0895E2
:1076AE00E695E695E170E295E07FEE0FEA2BAE2FC0
:1076BE000895E295E07FEA2BAE2FE52F0895E6952B
:1076CE00E695E69581CEEA2BAE2FDFCFE295EF70F1
:1076DE00E695E170EE0FEE0F0895E295EF70E695E8
:1076EE00E695E170EE0F0895E295E170C0CFFE01D0
:1076FE00E55AFF4FE0810895EA2BAE2FFE01E35AC3
:10770E00FF4FE0810895E295EF70E695E1700895E0
:10771E00FE01E65AFF4FE0810895EA2BAE2FF8CF17
:10772E00FE01E35AFF4FE0810895E295EF70E69572
:10773E00E6950895FE01E75AFF4FE0810895EA2B82
:10774E00AE2FFE01E25AFF4FE0810895EA2BAE2FD5
:10775E0097CFFE01E25AFF4FE0810895AE2FFE0152
:10776E00E05BFF4FE0810895E170EE0FEE0FEA2B24
:10777E000895E17057DCEA2B0895E695E170E295E5
:10778E00E07FEE0FEA2B0895E295E07FEA2BAE2F15
:10779E000895E695E695E8CFE170EE0FEA2BAE2F51
:1077AE000895FE01EF5AFF4FE0810895FE01EE5A53
:1077BE00FF4FE0810895FE01ED5AFF4FE0810895DD
:1077CE00289885E28A95F1F731E008955E9884E075
:1077DE008A95F1F7ECE0E31B089584E08A95F1F7C2
:1077EE005E9A84E08A95F1F708955D9A85E28A950E
:1077FE00F1F7289A85E28A95F1F7E2CF5E9884E058
:10780E008A95F1F70895EAE00E94353E0E2A089512
:10781E00109639F08DEC9AE00197F1F7A895119733
:10782E00C9F7089530976040704009F07058089578
:10783E00552342F4503811F4E0FF04C03196691F0D
:10784E00791F6BF050E8572711F45F93CFC05F3F5D
:10785E0031F0660F000C57956795752F08955F935D
:10786E0000200AF0CFC0C8C050E8192E1522880F8C
:10787E00991F9527550F879550E8072E0522660FFD
:10788E00771F7527550F67950895689401C0E89482
:10789E005F93F2DF703818F07F3F08F4A7C056E10F
:1078AE00571BAAF4519558300EF4593030F0EFEFC3
:1078BE00FFEF6FEF7FE777F91AC077275523B9F0FF
:1078CE00EE0FFF1F661F771F5A95D1F710C077274F
:1078DE00583028F0EF2FF62F672F5850F9CF552339
:1078EE0031F076956795F795E7955A95D1F7002083
:1078FE000AF45BD15F910895689401C0E8943097C3
:10790E0060407040B1F0002426F0772312F400940A
:10791E004CD1172E7EE1112032F07A95EE0FFF1F1B
:10792E00661F111CF9CFEF2FF62F612D5F938ADFA3
:10793E005F9108954F93AF01FD01DA01AB01BC01D8
:10794E00CA01402D012C142E4F910895EA0FFB1FF2
:10795E00681F0895E095F0956095EF5FFF4F6F4FAC
:10796E0008955F9381DF903871F150E8152604C0B9
:10797E005F937ADF903839F1703821F1572F591B08
:10798E002BF112F4D7DFFACF583118F0AA27BB2704
:10799E008827583028F0AB2FB82F88275850F9CFAA
:1079AE00552329F08695B795A7955A95D9F7502D59
:1079BE00512572F0CBDF38F46795F795E7957395FF
:1079CE0013F420C0B7DF3EDF5F910895D8F7FBCFE9
:1079DE00EA1BFB0B680B51F010F40094BBDF66231F
:1079EE0092F3EE0FFF1F661F7A95CBF7EE27FF2758
:1079FE00662777275F910895EFEFFFEF6FE77FEF31
:107A0E005F910895EFEFFFEF6FE77FE75F910895C6
:107A1E005F932ADF703851F3903841F301240894B4
:107A2E00791F23F41CF300203AF3ECCF0F921F932F
:107A3E002F933F934F93112722279927689FA001D9
:107A4E008F9F302D410D591F6B9F300D411D591FBA
:107A5E008E9F27D0BF9F25D06A9F23D0BE9F1DD05B
:107A6E00AF9F1BD0AE9F110D291F391F491F591FE4
:107A7E00E32FF42F652F522F4F913F912F911F918E
:107A8E000F9066232AF0550FEE1FFF1F661F02C0D0
:107A9E0073954BF2CDDE5F910895100D211D391FA8
:107AAE0002C0200D311D491F591F08955F93DCDE62
:107ABE00703821F411200AF49FCFA4CF903809F426
:107ACE0095CF01240894970B1BF4D4F30020F3CF29
:107ADE00792F1F932F933F934F9311241127222712
:107AEE0033274427552790E2AE17BF078607410775
:107AFE0030F0AE1BBF0B860B410B089401C088946F
:107B0E00551F221F331F111CAA1FBB1F881F441F86
:107B1E009A9551F7F901612D4F913F912F911F9138
:107B2E00662332F0550FEE1FFF1F661F7A9543F244
:107B3E007FDE5F91089599239AF0772342F097178D
:107B4E0048F029F4AE17BF07860720F031F098945D
:107B5E008894089598940894089518948894089594
:107B6E007723C2F7971798F3A9F7EA17FB07680769
:107B7E0088F399F3ECCFDFDFE1E009F008F0EE27B0
:107B8E000895D9DFE1E009F008F4EE270895EA0F31
:107B9E00FB1F681F791F0895AE1BBF0B860B970B3B
:107BAE000895F195E195F0400895F09560957095E2
:107BBE00E195FF4F6F4F7F4F0895EE230E2EEA2F64
:107BCE0019F0E6950A94E9F70895EE230E2EFD01BD
:107BDE0021F0EE0FFF1F0A94E1F70895EE230E2E0B
:107BEE00FD0121F0F695E7950A94E1F70895F695D3
:107BFE00E795F695E795F695E795F695E795089549
:107C0E00FE2FFF0FFF0B6F2F7F2F08956F2F660F25
:107C1E00660B762F08958B2F880F880B982F08955B
:107C2E00EA17E1E009F0EE270895EA17E1E009F41A
:107C3E00EE270895AE17E1E00CF4EE270895AE1787
:107C4E00E1E00CF0EE270895EA17E1E00CF0EE27E4
:107C5E000895AE17E1E008F4EE270895AE17E1E0BF
:107C6E0008F0EE270895EA17E1E008F0EE270895F0
:107C7E00EA17FB07E1E009F0EE270895EA17FB0784
:107C8E00E1E009F4EE270895AE17BF07E1E00CF02E
:107C9E00EE270895EA17FB07E1E00CF0EE270895B2
:107CAE00EA17FB07E1E008F4EE270895AE17BF07C9
:107CBE00E1E008F0EE270895EA17FB07E1E008F08F
:107CCE00EE270895EA17FB0768077907E1E009F048
:107CDE00EE270895EA17FB0768077907E1E009F434
:107CEE00EE270895EA17FB0768077907E1E00CF421
:107CFE00EE270895AE17BF0786079707E1E00CF051
:107D0E00EE270895EA17FB0768077907E1E00CF004
:107D1E00EE270895FA9FF02DEB9FF00DEA9FE02DD0
:107D2E00F10D08957A9F702D6B9F700DF89F700D59
:107D3E00E99F700D6A9F602D710DFB9F600D711D87
:107D4E00E89F600D711D8827FA9FF02D610D781F39
:107D5E00EB9FF00D611D781FEA9FE02DF10D681F5E
:107D6E00781F08956E2F6A9FF0016B9FF00D089596
:107D7E0074D0D0DF0EF415DF08957DD0D3DF0EF46E
:107D8E0014DF08950024112490E1AA0FBB1F001CDC
:107D9E00111C0E1A1F0A18F40E0E1F1E01C0A16030
:107DAE009A9599F7FD01D001089557D0EBDF0EF4A7
:107DBE00F8DE08953F934F935F93002411244427D8
:107DCE00552730E2AA0FBB1F881F991F001C111CDC
:107DDE00441F551F0E1A1F0A460B570B28F40E0E82
:107DEE001F1E461F571F01C0A1603A9559F7FD018E
:107DFE00BC01D001CA015F914F913F9108953BD0D4
:107E0E00D9DF0EF4D2DE0895BDDFFD010895E894AA
:107E1E00B7FF04C0A095B09511966894F7FDC1DE2A
:107E2E00B1DFFD010EF4BDDE0895C4DFFD01BC011E
:107E3E000895E89497FF09C0A095B0958095909508
:107E4E00AF5FBF4F8F4F9F4F689477FDAEDEB2DFAF
:107E5E00FD01BC010EF4A9DE0895E894F7FF02C0FF
:107E6E00A0DE6894B7FF06C0A095B095119600F8F5
:107E7E00039400FA0895E89477FF02C096DE6894A2
:107E8E0097FF0BC00024A095B09580959095119604
:107E9E00801D901D00F8039400FA0895ED91FC9159
:107EAE0011970895ED93FD936D937C930895E8815A
:107EBE00F9816A817B810895A881B9818A819B812C
:107ECE000895E883F9836A837B830895E883E983C1
:107EDE00EA83EB830895689401C0E89401D00FDD26
:107EEE00182E862F612D192E972F712D1B2EBF2F19
:107EFE00F12D1A2EAE2FE12D0895129602D0BF014C
:107F0E001297119602D0FE2F1197F999FECFFF937B
:107F1E00FFB7F894A1BDB2BDF89AE0B5FFBFFF91CF
:107F2E00089507D012960F01FB0103D0F0011297AE
:107F3E00089507D01196EF93EF2F03D0EF9111977D
:107F4E000895F99B02C0A895FCCF9FB7F894A1BDE8
:107F5E00B2BDF89A80B5E81719F0E0BDFA9AF99A11
:107F6E009FBF089500240E160F06060607060895F5
:107F7E0000240A160B06089500240A160B0608069E
:107F8E0009060895EA17FB07680779070895AE17E3
:107F9E00BF07860797070895E894EE2309F06894C3
:107FAE000895AC0FBD1F05900D928A95E1F70895C7
:00000001FF
